:100000000C94A20E0C94E90E0C94E90E0C94E90EDB
:100010000C94E90E0C94E90E0C94E90E0C94E90E84
:100020000C94E90E0C94E90E0C9471200C942D2084
:100030000C94ED2B0C94E90E0C94E90E0C94E90E43
:100040000C94E90E0C94E90E0C94E90E0C94E90E54
:100050000C94E90E0C944E210C94E90E0C94E90ECC
:100060000C94E90E0C94E90E0C94E90E0C94E90E34
:100070000C94E90E0C94E90E0C94E90E0C94E90E24
:100080000C94E90E0C94E90E0C94E90E0C94E90E14
:100090000C94E90E0C94E90E0C94E90E0C94E90E04
:1000A0000C94E90E0C94E90E0C94E90E05010980FC
:1000B000A101850319012AB700150126B700950192
:1000C00075108100C0050C0901A101850419012AE0
:1000D000A002150126A002950175108100C005013E
:1000E0000906A1018506050719E029E71500250184
:1000F0009508750181020507190029EF15002501F2
:1001000095F075018102050819012905950575010C
:100110009102950175039101C00660FF0961A1017B
:100120000962150026FF00952075088102096315F4
:100130000026FF00952075089102C005010906A15F
:1001400001050719E029E7150025019508750181CA
:10015000029501750881010507190029FF15002680
:10016000FF00950675088100050819012905950508
:1001700075019102950175039101C0000000000016
:1001800000E0CE9CF8FCFE80E020000000000000B3
:10019000000000000000000000000000000000005F
:1001A000000000008080C0C0E0E0F0F0F8FCFEFC41
:1001B000F8F0E0E0C0C08080800000000000000097
:1001C000000000000000000000000000000000002F
:1001D000000000000000000000000000000000001F
:1001E000000000000000000000000000000000000F
:1001F00000000000000000000000000101010102F9
:100200000238F7F7F7F7F7F7310008101010102051
:10021000202020404040408080F0F8DC363EEEFC5C
:10022000E09CFEFFFFFFFFFFCFCFFFFFBF7F7FBF41
:10023000FFFF7FFFFFFFFFFFFFFFFFFFFEFEFCFC56
:10024000FCFCFEFEFFFFFF3F00000000808000007E
:10025000000000000000000000000000000000009E
:10026000000000000000000000000000000000008E
:10027000000000000000000000000000000000007E
:10028000000003070F0F0F01000000000000000036
:1002900080C0E030382C44C4C4687859899191D327
:1002A000F3A3232727C7C74F4F8F8F9F9F1F1F3F42
:1002B0003E3E3F7F7F7F7FFCFCFFFFFFFFFFFFFF96
:1002C000FFFFFFFFFFFFFEF8E000003F1F0783C0B6
:1002D000E0E0C0000000000000000000000000009E
:1002E000000000000000000000000000000000000E
:1002F000000000000000000000000000000000807E
:10030000C0603010180808081810306040C0868798
:1003100085C449693E0E131113123C2C26274568EB
:1003200078589D9793E362343C2C26C7C5693919E8
:100330001D36A2E26224183C7E7F7F7FBF3F1F1FD5
:100340008FE76327274747CFCF0F081010111121E0
:100350002323214040404080808080000000000036
:10036000000000000000000000000000000000008D
:10037000000000000000000000000000000000007D
:100380000000000000000000000000000000E0CEBF
:100390009CF8FCFE80E0200000000000000000004F
:1003A000000000000000000000000000000000004D
:1003B000008080C0C0E0E0F0F0F8FCFEFCF8F0E067
:1003C000E0C0C0808080000000000000000000004D
:1003D000000000000000000000000000000000001D
:1003E000000000000000000000000000000000000D
:1003F00000000000000000000000000000000000FD
:10040000000000000000000001010101020238F7B5
:10041000F7F7F7F7F731000810101010A0A0202010
:1004200040464F5F9F9C9080C0E0F0F8F8FCFCFED7
:10043000FFFFFFFFFFCFCFFFFFBF7F7FBFFFFF7F2C
:10044000FFFFFFFFFFFFFFFFFF7EBEBCBC7CFCFE8B
:10045000FEFFFFFF3F000000000000000000000062
:10046000000000000000000000000000000000008C
:10047000000000000000000000000000000000007C
:100480000000000000000000000000000000000369
:10049000070F0F0F01000000000000070F8FC7E3D8
:1004A00031382C0464F8FEFFFFFFFFFF7FBF8F276A
:1004B0002727C7C74F4F8F8F9F9F1F1F3F3E3E3F2E
:1004C0007F7F7F7FFCFCFF81FAFFE6E7FDFFFCF307
:1004D000FFFFFFFEF8E00000000000000000000049
:1004E000000000000000000000000000000000000C
:1004F00000000000000000000000000000000000FC
:1005000000000000000000000000000080C060301B
:1005100010180808081810306040C0868785C44944
:10052000693E0E131112123D2D2526446878589D00
:100530009793E362343C2C26C7C56939191D36A24E
:10054000E262343C2C44C8C8E9B911111393E36347
:1005500027274747CFCF0F0810101010202020204A
:10056000404040408080808000000000000000008B
:10057000000000000000000000000000000000007B
:10058000000000000000000000000000000000006B
:100590000000000000000000000000E0CE9CF8FC1D
:1005A000FE80E020000000000000000000000000CD
:1005B000000000000000000000000000000080803B
:1005C000C0C0E0E0F0F0F8FCFEFCF8F0E0E0C0C0F5
:1005D000808080000000000000000000000000009B
:1005E000000000000000000000000000000000000B
:1005F00000000000000000000000000000000000FB
:1006000000000000000000000000000000000000EA
:10061000000000000001010101020238F7F7F7F7BE
:10062000F7F7310008101010102020202040404023
:10063000408080F0F8DC363EEEFCE09CFEFFFFFFE1
:10064000FFFFCFCFFFFFBF7F7FBFFFFF7FFFFFFF1A
:10065000FFFFFFFFFFFF7EBEBCBC7CFCFEFEFFFF7A
:10066000FF3F00000000000000000000000000004C
:10067000000000000000000000000000000000007A
:10068000000000000000000000000000000000006A
:1006900000000000000000000000000003070F0F32
:1006A0000F01000000000000000080C0E030382C86
:1006B00044C4C4687859899191D3F3A3232727C7E9
:1006C000C74F4F8F8F9F9F1F1F3F3E3E3F7F7F7FB4
:1006D0007FFCFCFF81FAFFE6E7FDFFFCF3FFFFFF75
:1006E000FEF8E00000000000000000000000000034
:1006F00000000000000000000000000000000000FA
:1007000000000000000000000000000000000000E9
:1007100000000000000000000080C06030101808D9
:1007200008081810306040C0868785C449693E0EAD
:10073000131113123C2C2627456878589D9793E394
:1007400062343C2C26C7C56939191D36A2E26234D1
:100750003C2C44C8C8E9B911111393E36327274718
:1007600047CFCF0F0810101010202020204040400D
:100770004080808080000000000000000000000039
:100780000000000000000000000000000000000069
:100790000000000000000000000000000000000059
:1007A0000000000000000000E0CE9CF8FCFE80E0AD
:1007B0002000000000000000000000000000000019
:1007C00000000000000000000000008080C0C0E0C9
:1007D000E0F0F8FCFEFFFEFCF8E0E0E0E0E0C0C086
:1007E000C080800000000000000000000000000049
:1007F00000000000000000000000000000000000F9
:1008000000000000000000000000000000000000E8
:1008100000000000000000000000000000000000D8
:10082000000001010101020238F7F7F7F7F7F7318D
:1008300000081010101020202020404040408080F0
:100840008080C0E0F0F8F8FCFCFEFFFFFFFFFFCF68
:10085000CFFFFFBF7F7FBFFFFF7FFFFFFFFFFFFFD8
:10086000FFFFFFFEFEFCFCFCFCFEFEFFFFFF3F0067
:100870000000000000000000000000000000000078
:100880000000000000000000000000000000000068
:100890000000000000000000000000000000000058
:1008A00000000000000000000003070F0F0F010010
:1008B0000000000000000080C0E030382C0464F824
:1008C000FEFFFFFFFFFF7FBF8F272727C7C74F4FC1
:1008D0008F8F9F9F1F1F3F3E3E3F7F7F7F7FFCFC90
:1008E000FFFFFFFFFFFFFFFFFFFFFFFFFFFEF8E03F
:1008F00000000000000000000000000000000000F8
:1009000000000000000000000000000000000000E7
:1009100000000000000000000000000000000000D7
:1009200000000000000080C060301018080808189F
:1009300010306040C0868785C449693E0E1311128D
:10094000123D2D2526446878589D9793E362343CE8
:100950002C26C7C56939191D36A2E26224183C7ECF
:100960007F7F7FBF3F1F1F8FE76327274747CFCF7B
:100970000F081010101020202020404040408080A0
:100980008080000000000000000000000000000067
:100990000000000000000000000000000000000057
:1009A0000000000000000000000000000000000047
:1009B0000000000000E0CE9CF8FCFE80E02000007B
:1009C0000000000000000000000000000000000027
:1009D000000000000000000000008080C0E0F0F88F
:1009E000FCFEFFFEFCF8F0E0C0C0C080800000000C
:1009F00000000000000000000000000000000000F7
:100A000000000000000000000000000000000000E6
:100A100000000000000000000000000000000000D6
:100A200000000000000000000000000000000001C5
:100A3000010101020238F7F7F7F7F7F73100081064
:100A4000101010202020204040404080808080C036
:100A5000E0E0F0F0F8F8FCFCFEFFFFFF9F9FFFFFD7
:100A60007FFFFF7FFFFFFFFFFFFFFFFFFFFFFFFF96
:100A7000FEFEFCFCFCFCFEFEFFFFFF3F0000000052
:100A80000000000000000000000000000000000066
:100A90000000000000000000000000000000000056
:100AA0000000000000000000000000000000000046
:100AB00000000000000003070F0F0F0100000000FE
:100AC0000000000080C0E030382C0464F8FEFFFF16
:100AD000FFFFFF7FBF8F272727C7C74F4F8F8F9FEE
:100AE0009F1E1E3F3D3D3E7F7F7F7FF9F9FFFFFF49
:100AF000FFFFFFFFFFFFFFFFFFFFFCF0C000000054
:100B000000000000000000000000000000000000E5
:100B100000000000000000000000000000000000D5
:100B200000000000000000000000000000000000C5
:100B300000000080C06030101808080818103060ED
:100B400040C0868785C449693E0E131112123D2D9F
:100B50002526446878589D9793E362343C2C26C739
:100B6000C56939191D36A2E26224183C7E7F7F7F59
:100B7000BF3F1F1F8FE76327274747CFCF0F0810BF
:100B800010101020202020404040408080808000B5
:100B90000000000000000000000000000000000055
:100BA0000000000000000000000000000000000045
:100BB0000000000000000000000000000000000035
:100BC0000000E0CE9CF8FCFE80E020000000000069
:100BD0000000000000000000000000000000000015
:100BE00000000000000000008080C0E0F0F8FCFE83
:100BF000FCF8F0E0C0C080808080000000000000B1
:100C000000000000000000000000000000000000E4
:100C100000000000000000000000000000000000D4
:100C200000000000000000000000000000000000C4
:100C300000000000000000000000000001010101B0
:100C4000020238F7F7F7F7F7F73100081010101025
:100C5000202020204040404080808080C0E0E0F0A4
:100C6000F0F8F8FCFCFEFFFFFF9F9FFFFF7FFFFFF8
:100C70007FFFFFFFFFFFFFFFFFFFFFFFFEFCFCF812
:100C8000F8F8F8FCFCFEFEFE7E000000000000000C
:100C90000000000000000000000000000000000054
:100CA0000000000000000000000000000000000044
:100CB0000000000000000000000000000000000034
:100CC00000000003070F0F0F0100000000000000EC
:100CD0000080C0E030382C0464F8FEFFFFFFFFFF07
:100CE0007FBF8F272727C7C74F4F8F8F9F9F1E1EFE
:100CF0003F3D3D3E7F7F7F7FF9F9FFFFFFFFFFFF15
:100D0000FFFFFFFFFFFFFFFCF0C00000000000003E
:100D100000000000000000000000000000000000D3
:100D200000000000000000000000000000000000C3
:100D300000000000000000000000000000000000B3
:100D400080C0603010180808081810306040C08655
:100D50008785C449693E0E131112123D2D25264484
:100D60006878589D9793E362343C2C26C7C569394F
:100D7000191D36A2E26224183C7E7F7F7FBF3F1F91
:100D80001F8FE76327274747CFCF0F08101010109A
:100D900020202020404040408080808000000000D3
:100DA0000000000000000000000000000000000043
:100DB0000000000000000000000000000000000033
:100DC000000000000000000000000000000000E043
:100DD000CE9CF8FCFE80E020000000000000000037
:100DE0000000000000000000000000000000000003
:100DF00000000000008080C0E0F0F8FCFEFCF8F08D
:100E0000E0C0C08080808000000000000000000082
:100E100000000000000000000000000000000000D2
:100E200000000000000000000000000000000000C2
:100E300000000000000000000000000000000000B2
:100E40000000000000000000000101010102023862
:100E5000F7F7F7F7F7F731000810101010202020EF
:100E6000204040404080808080C0E0F0F8F8FCFCEA
:100E7000FCFEFEFFFFFFCFCFFFFFBF7F7FBFFFFF67
:100E80007FFFFFFFFFFFFFFFFFFEFCFCF8F8F8F815
:100E9000F8FCFCFCFC3C1C00000000000000000012
:100EA0000000000000000000000000000000000042
:100EB0000000000000000000000000000000000032
:100EC0000000000000000000000000000000000022
:100ED00003070F0F0F01000000000000000080C09A
:100EE000E030382C0464F8FEFFFFFFFFFF7FBF8F68
:100EF000272727C7C74F4F8F8F9F9F1F1F3F3E3EFC
:100F00003F7F7F7F7FFCFCFFFFFFFFFFFFFFFFFFB7
:100F1000FFFFFFFFFEF8E0000000000000000000FF
:100F200000000000000000000000000000000000C1
:100F300000000000000000000000000000000000B1
:100F40000000000000000000000000000080C06001
:100F50003010180808081810306040C0868785C413
:100F600049693E0E131112123D2D2526446878580A
:100F70009D9793E362343C2C26C7C56939191D3609
:100F8000A2E26224183C7E7F7F7FBF3F1F1F8FE756
:100F90006327274747CFCF0F0810101010202020BD
:100FA0002040404040808080800000000000000021
:100FB0000000000000000000000000000000000031
:100FC0000000000000000000000000000000000021
:100FD000000000000000000000000000E0CE9CF8CF
:100FE000FCFE80E020000000000000000000000087
:100FF0000000000000000000000000000000008071
:1010000080C0C0E0E0F0F8FCFEFFFEFCF8E0E0E0AD
:10101000E0E0C0C0C08080000000000000000000D0
:1010200000000000000000000000000000000000C0
:1010300000000000000000000000000000000000B0
:1010400000000000000000000000000000000000A0
:1010500000000000000001010101020238F7F7F76B
:10106000F7F7F73100081010101020202020404022
:10107000404080808080C0E0F0F8F8FCFCFEFFFF7C
:10108000FFFFFFCFCFFFFFBF7F7FBFFFFF7FFFFFD0
:10109000FFFFFFFFFFFFFFFEFEFCFCFEFEFEFFFF6B
:1010A000FFFF3F0F060000000000000000000000EE
:1010B0000000000000000000000000000000000030
:1010C0000000000000000000000000000000000020
:1010D0000000000000000000000000000003070FF7
:1010E0000F0F01000000000000000080C0E0303859
:1010F0002C0464F8FEFFFFFFFFFF7FBF8F27272729
:10110000C7C74F4F8F8F9F9F1F1F3F3E3E3F7F7F21
:101110007F7FFCFCFFFFFFFFFFFFFFFFFFFFFFFFE5
:10112000FFFEF8E0000000000000000000000000EA
:1011300000000000000000000000000000000000AF
:10114000000000000000000000000000000000009F
:101150000000000000000000000080C06030101897
:101160000808081810306040C0868785C449693E69
:101170000E131112123D2D2526446878589D979321
:10118000E362343C2C26C7C56939191D36A2E262D8
:1011900024183C7E7F7F7FBF3F1F1F8FE763272779
:1011A0004747CFCF0F0810101010202020204040BC
:1011B00040408080808000000000000000000000AF
:1011C000000000000000000000000000000000001F
:1011D000000000000000000000000000000000000F
:1011E00000000000000000000000000000000000FF
:1011F00000000000000000000000000000000000EF
:10120000000000000000007E0F00D4FFFFFFC700B9
:1012100000007800000000000000002A2B280000D9
:101220000000000000000000000000000000290095
:101230000000002C1E3420212224342627252E369F
:101240002D3738271E1F202122232425263333360D
:101250002E37381F0405060708090A0B0C0D0E0F60
:10126000101112131415161718191A1B1C1D2F31E3
:1012700030232D350405060708090A0B0C0D0E0F47
:10128000101112131415161718191A1B1C1D2F31C3
:1012900030354C00DA0281FFD9F1DB20A4A62EAF55
:1012A00000A0C000A1C800AED580A81FD300408D0B
:1012B000142000000000000000000080C0E0F0F0FA
:1012C000F87878383C3C3C3C38F8F8F8F0783C1E2C
:1012D0000F070300000000000000000080C0C0C035
:1012E000E0E0E0E0E0C0C0C08000000000000000DE
:1012F00000000000000000000000000000000000EE
:1013000000000000000000000000000000000000DD
:1013100000000000C0C0C00000000000000000008D
:1013200000000000000000000000000000000000BD
:101330000000000000000000F0FEFFFF0F070100AA
:10134000E0F0F8F8FCFC3C1E8FC7E3E10000071F4B
:10135000FFFFFCE00000000000F8FEFF0F030101AA
:1013600000E0E0E0E0E1E1E3E7E7E60080E0F070E4
:101370003838383870F0E08000C0E0F07038383825
:10138000383870F0E0C00080E0F0703838383870DD
:10139000F0E08000FFFFFF00C0E0F0703838383820
:1013A0003870F0E0C000F8F8F8F070383838000015
:1013B0000000000000000000073F7FFFF860000011
:1013C000070F1F1F3F3F3F3F1F1F0F0780C0E0F861
:1013D000FF7F3F07000000000001070F1F3C383867
:1013E000707070707038383C1F0F0700071F3F384F
:1013F00070707070383F1F0700FFFFFF0060606073
:101400006070783F1F0F00071F3F38707070703892
:101410003F1F07007F7F7F000F3F7F787060606015
:1014200060007F7F7F007F7F7F0000000000000062
:10143000000000000000000000C0E0F0783C1E0F3B
:101440000F1E1E1E1E1C1C1E1E1E1E0F0F07070336
:10145000010000000000000000000000000000008B
:10146000000000000000000000000000000000007C
:101470000000000000000000000F0F0F000000003F
:10148000000000000000000000000000000000005C
:10149000000000000000000000000000000000004C
:1014A000000000000000000000000000000000003C
:1014B000000000000000000000000000000000002C
:1014C00020202020005343524C00202020200043A5
:1014D0004150530057504D3A0000010101010101F4
:1014E00001010102020202020202020203030303DB
:1014F00003030303040404040404040505050505AB
:101500000606060606070707070708080808090968
:1015100009090A0A0A0B0B0B0C0C0C0D0D0D0E0E13
:101520000E0F0F0F101011111112121313141415A6
:101530001516161717181819191A1A1B1B1C1D1D1A
:101540001E1E1F2020212222232424252626272870
:1015500029292A2B2C2D2D2E2F30313232333435A0
:10156000363738393A3B3C3D3E3F404142434445A3
:10157000464748494A4C4D4E4F5051535455565882
:10158000595A5B5D5E5F616264656668696B6C6D2C
:101590006F7072737577787A7B7D7E8082838587A2
:1015A000888A8C8E8F91939596989A9C9EA0A2A3E0
:1015B000A5A7A9ABADAFB1B3B5B7BABCBEC0C2C4E5
:1015C000C6C9CBCDCFD1D4D6D8DBDDDFE2E4E7E9A5
:1015D000EBEEF0F3F5F8FAFDFF00AF00AE29003AAC
:1015E000003B003C003D003E003F00400041004207
:1015F0000043004400450000004600470048003515
:10160000001E001F002000210022002300240025CE
:1016100000260027002D002E002A0049004A004B1A
:10162000002B0014001A000800150017001C0018F9
:10163000000C00120013002F00300031004C004D50
:10164000004E00390004001600070009000A000BD4
:10165000000D000E000F00330034000000280000D1
:101660000000000000E10064001D001B00060019DE
:1016700000050011001000360037003800E500E5D5
:1016800000000052000000E000E300E20000000063
:10169000002C000000000000000000E6000151E402
:1016A000000000500051004F00A600D55C680069A2
:1016B000006A006B00B900B80001000100010001E0
:1016C00000DE5C00000100AA00A900010001000189
:1016D0000001000100010001000100010001000102
:1016E00000010001000100C55CC75CCB5C0100018A
:1016F00000010001000100010001000100010001E2
:10170000000100010001000100C65CC85CCC5C0166
:1017100000010001000100010001000100010001C1
:10172000000100010001000000C25C000000000098
:10173000000100010001000100B2000100010001F0
:10174000000100010001000100010001000000C9CA
:101750005C00000100010001000000000001000029
:10176000000000000000000100010001000000C4B2
:101770005CCA5CC35C09025B00030100A0FA0904B7
:1017800000000103010100092111010001224000B4
:10179000070581030800010904010002030000009D
:1017A0000921110100012222000705820320000106
:1017B00007050303200001090402000103000000E3
:1017C000092111010001226D000705840320000199
:1017D00012010002000000080700070001000102DA
:1017E00000010A03470047003800360000001003DC
:1017F00047006F0070006F006C0061007200000015
:101800000403090407087F0807003E5B4F5B3E00A6
:101810003E6B4F6B3E001C3E7C3E1C00183C7E3CE9
:1018200018001C577D571C001C5E7F5E1C000018B2
:101830003C180000FFE7C3E7FF0000182418000071
:10184000FFE7DBE7FF0030483A060E00262979293A
:101850002600407F05050700407F05253F002A1C24
:10186000771C2A007F3E1C1C0800081C1C3E7F00C1
:1018700014227F2214005F5F005F5F0006097F0172
:101880007F00006689956A0060606060600094A2D5
:10189000FFA2940008043E04080008103E1008004F
:1018A00008082A1C0800081C2A0808001E1010102E
:1018B00010000C1E0C1E0C0030383E383000060E96
:1018C0003E0E060000000000000000005F00000067
:1018D000000700070000147F147F1400242A7F2AC9
:1018E0001200231308646200364956205000000895
:1018F00007030000001C224100000041221C0000E0
:101900002A1C7F1C2A0008083E080800008070304E
:1019100000000808080808000000606000002010AF
:10192000080402003E5149453E0000427F4000004D
:101930007249494946002141494D33001814127F2C
:1019400010002745454539003C4A494931004121AD
:1019500011090700364949493600464949291E0000
:1019600000001400000000403400000000081422B1
:101970004100141414141400412214080000020140
:10198000590906003E415D594E007C1211127C003F
:101990007F49494936003E41414122007F41414152
:1019A0003E007F49494941007F09090901003E4144
:1019B000415173007F0808087F0000417F4100000B
:1019C0002040413F01007F08142241007F404040F9
:1019D00040007F021C027F007F0408107F003E4110
:1019E00041413E007F09090906003E4151215E0048
:1019F0007F091929460026494949320003017F0120
:101A000003003F4040403F001F2040201F003F4058
:101A100038403F0063140814630003047804030093
:101A20006159494D4300007F4141410002040810C3
:101A30002000004141417F000402010204004040B7
:101A40004040400000030708000020545478400044
:101A50007F2844443800384444442800384444280B
:101A60007F0038545454180000087E09020018A45E
:101A7000A49C78007F080404780000447D400000A6
:101A80002040403D00007F102844000000417F407E
:101A900000007C04780478007C0804047800384452
:101AA00044443800FC182424180018242418FC008E
:101AB0007C080404080048545454240004043F449F
:101AC00024003C4040207C001C2040201C003C4066
:101AD00038403C004428102844004C9090907C00F2
:101AE0004464544C44000008364100000000770074
:101AF00000000041360800000201020402003C26FA
:101B000023263C00103810101C000C7A417A0C007F
:101B1000182F412F1800227222272200081C0808C3
:101B20000800080838202828000000000000002ACB
:101B30002A2A00004E464A502F003E4555513E008D
:101B400048507E5048003E4971493E0010224F20C7
:101B500010000E060A10200020100A060E000808C9
:101B6000081C080000000000000000000000000049
:101B70000000000000000000000000000000000065
:101B80000000E0F0F0F0E0ECEEF7F37020007C7C79
:101B90007C7E007E7E7E7F7F7F000080C0E07E5B5B
:101BA0004F5BFEC00000C000DCD7DEDEDED7DC000D
:101BB000C000000000000000000000000000000065
:101BC0000000000000000000000000000000000015
:101BD0000000000000000000000000000000000005
:101BE00000000000000000000000000000000000F5
:101BF00000000000000000000000000000000000E5
:101C000000000000000000000000000000000000D4
:101C100000000000000000000000000000000000C4
:101C200000000000000000000000000000000000B4
:101C300000000000000000000000000000000000A4
:101C400000000F1F3F7F7F7F7F7F3F1E0C001F1F05
:101C50001F3F003F3F3F7F7F7F00307B7F783020FA
:101C60002030787F3B0003000F7F0F0F0F7F0F00A6
:101C70000300000000000000000000000000000061
:101C80000000000000000000000000000000000054
:101C90000000000000000000000000000000000044
:101CA0000000000000000000000000000000000034
:101CB0000000000000000000000000000000000024
:101CC0000000000000000000000000000000000014
:101CD0000000000000000000000000000000000004
:101CE00000000000000000000000000000000000F4
:101CF00000000000000000000000000000000000E4
:101D000000000000000000000000000000000000D3
:101D100000000000000000000000000000000000C3
:101D200000000000000000000000000000000000B3
:101D300000000000000000000000000000000000A3
:101D40000000000011241FBECFEFDAE0DEBFCDBFE0
:101D500004B603FE27C08091EF079091F007A09191
:101D6000F107B091F2078730904BA740B04BD1F408
:101D70001092EF071092F0071092F1071092F207FD
:101D800014BE84B7877F84BF0FB6F894A89580915E
:101D90006000886180936000109260000FBEE0E0F8
:101DA000F8E3099513E0A0E0B1E0EEECFDE602C037
:101DB00005900D92A831B107D9F727E0A8E1B3E06B
:101DC00001C01D92AF3EB207E1F70E94102C0C94A7
:101DD000A1360C940000CF93DF934091ED07509112
:101DE000EE074D5E55409A01235F3D4F2130324052
:101DF000C0F020E032E0241B350B6091EB057091C0
:101E0000EC05FC01CA01240F351FC1E0D0E08217A8
:101E1000930750F07093EC056093EB05DF91CF9141
:101E200008952DE032E0E9CF4491DC01A351BA4F8F
:101E30005C91451781F04C93AC01A5E05695479510
:101E4000AA95E1F7DE0102C0AA0FBB1F4A95E2F78F
:101E5000AD016A2B752B01963196D9CF9091DD0596
:101E6000937061F081110BC094609093DD05109226
:101E70001B018091DC0581608093DC0508958D3025
:101E800010F09063F2CF880F880F982BEECF9091CF
:101E9000DD05937071F08093DE056093DF05493CAA
:101EA00008F048EC4093E0058091DC058160809368
:101EB000DC050895E8EDF0E080818E7F808310924C
:101EC000E2001092DA001092E100A0EEB0E08C91F6
:101ED00081608C9380818F77808319BCA7EDB0E0FF
:101EE0008C918E7F8C9380818F7E80831092A6054B
:101EF00008952091E4003091E50095E6A901209134
:101F0000EC00822F817020FF06C08091E80080FFE6
:101F100006C080E008952091E80022FD1AC080915B
:101F2000CB05882389F0853089F08091EB0085FD11
:101F30000FC02091E4003091E50042175307F9F2F9
:101F40009150E1F684E0089582E0089583E00895D9
:101F500081E00895EF92FF920F931F93CF937C013E
:101F60008B010E94790FC82F811117C08091E80062
:101F700085FD0BC08091E8008E778093E8000E9479
:101F8000790F882399F3C82F08C0F70181917F0149
:101F90008093F1000150110949F78C2FCF911F91C7
:101FA0000F91FF90EF9008958091CD0587FF13C0AA
:101FB0008091E80082FF06C08091E8008B778093D3
:101FC000E80004C08091CB058111F2CF0895809183
:101FD000CB058823D9F38091E80080FFF8CF80916A
:101FE000E8008E77ECCF982F9093E900242F762F7E
:101FF00050E0891731F07091EC002091ED00509184
:10200000F00021FD07C09F5F973071F78093E900D2
:1020100081E008953091EB003E7F3093EB003091EA
:10202000ED003D7F3093ED003091EB003160309357
:10203000EB007093EC002093ED005093F0002091A2
:10204000EE0027FDE0CF80E00895CF92DF92EF927F
:10205000FF920F931F93CF93DF93C8EDD0E0888159
:102060008F7E8883E7EDF0E080818160808384E06B
:1020700082BF81E08093A60588818E7F888302EEEF
:1020800010E0F80110821092DA0081EEC82ED12CF7
:10209000F601108288818F778883888180688883A1
:1020A00088818F7D888319BC1092CB051092CC0556
:1020B0001092CA051092C90590EEE92EF12CF70195
:1020C00080818B7F808388818160888342E060E0AB
:1020D00080E00E94F30FF60180818E7F8083F801FB
:1020E000808181608083808188608083F701808126
:1020F0008E7F8083888180618883DF91CF911F915B
:102100000F91FF90EF90DF90CF900895FC018091A8
:10211000D3059091D40586179707A0F06115710536
:1021200029F49091E8009E779093E80090E0611583
:10213000710551F4911108C08091E80082FF34C00C
:1021400080E00895BC01F2CF8091CB058823C1F1D6
:102150008530C1F18091E80083FD30C08091E800B6
:1021600082FDEACF8091E80080FFE1CF8091F3000B
:102170002091F200382F6115710519F028303105D2
:1021800058F091E02830310509F090E02091E80006
:102190002E772093E800CBCF81918093F10061509E
:1021A00071092F5F3F4FE7CF8091CB05882341F026
:1021B000853041F08091E80083FFBECF81E0089533
:1021C00082E0089583E00895089508958091A80518
:1021D0000895CF92DF92EF92FF922FB7F894C090BC
:1021E0009D05D0909E05E0909F05F090A0052FBF23
:1021F000A7019601261B370B480B590BCA01B901E1
:10220000FF90EF90DF90CF9008952FB7F8946091F2
:102210009D0570919E0580919F059091A0052FBF0F
:102220000895209117012223C9F02091A10527FFCD
:1022300015C0E62FE695E695E695EE31D8F4E80F61
:10224000F92FF11D677021E030E001C0220F6A957F
:10225000EAF720958281282322830895FC01329693
:1022600008962191621303C0DF0111971C92E817B1
:10227000F907B9F70895209117012223C1F02091A1
:10228000A10527FF14C0E62FE695E695E695EE3109
:10229000F8F4E80FF92FF11D677021E030E001C07C
:1022A000220F6A95EAF78281822B82830895FC01CE
:1022B00032962FEF30E04191641751F02F3F19F41F
:1022C000411101C0232F3F5F3630A9F72F3F09F49A
:1022D0000895820F911D27FD9A95FC016283089550
:1022E00020919B0530919C052817390771F0909338
:1022F0009C0580939B05E0919905F0919A05309794
:1023000021F00084F185E02D09940895209197052E
:10231000309198052817390771F0909398058093AC
:102320009705E0919905F0919A05309721F0068084
:10233000F781E02D09940895E0919905F0919A05AF
:10234000309721F00190F081E02D099480E008950C
:102350002091E40536E0839FC0011124629F800D27
:10236000911D1124811522E0920714F090E080E085
:1023700083519A4F9093EE078093ED070895FA01E9
:10238000811101C0FB010994E5E6F4E081836083DB
:102390004283339695E0E139F907C1F70895FC01CE
:1023A000EE0FFF1FE80FF91FEB59FB4F61834083CE
:1023B00022830895FC019B01AC0197FF04C04427D0
:1023C0005527481B590BBA01620F731F37FD0FC009
:1023D000241B350BC901A5E0880F991FAA95E1F7C9
:1023E0000E94F53380E2861BF7FD81950895CB01AD
:1023F00065E0880F991F6A95E1F7BA01621B730BBC
:102400000E94F53380E6EFCFEDEDF5E0248130E179
:10241000231B08F420E024838091DC0581608093F5
:10242000DC050895EDEDF5E0248130E1230F08F49B
:102430002FEF24838091DC0581608093DC05089573
:10244000EDEDF5E0438120E1421B08F440E081819D
:10245000628190E00C94470FEDEDF5E0438120E1BF
:10246000420F08F44FEF8181628190E00C94470F96
:10247000EDEDF5E0628120E1621B08F460E081810E
:10248000438190E00C94470FEDEDF5E0628120E18F
:10249000620F08F46FEF8181438190E00C94470F45
:1024A000EDEDF5E08181438162818850990B0C94B8
:1024B000470FEDEDF5E0818190E043816281089660
:1024C0000C94470F8091DD0586958695815009F41F
:1024D0008CE00C942E0F8091DD05869586958F5F9C
:1024E0008D3008F081E00C942E0F0C94C4110C94E4
:1024F000CF110F931F9310E0F801EE0FFF1FE4516F
:10250000FE4F9081905797FD9195000F111FF80194
:10251000E351FE4F00810052110B2003F001219F77
:10252000F00D112408E310E0091B110997FD139524
:1025300040039001419F300D1124E20FF31F9F01D2
:10254000220F331F2E0F3F1F37FF02C021583F4F6E
:10255000220F232F221F330B620F1F910F9108951B
:102560000F931F93522F10E0F801EE0FFF1FE3515E
:10257000FE4FA081A052BB0B9D015203F001539F5F
:10258000F00D1124000F111FD801A451BE4F0C9162
:102590000057110B40039001419F300D11242E0F65
:1025A0003F1F37FF02C0215C3F4F96E035952795CE
:1025B0009A95E1F7620F1F910F9108950F931F9362
:1025C000522F10E0F801EE0FFF1FE351FE4FA081E4
:1025D000A052BB0B9D015203F001539FF00D11243B
:1025E000000F111FD801A451BE4F0C910057110BC1
:1025F00040039001419F300D11242E0F3F1F37FFE4
:1026000002C021583F4F220F232F221F330B620F8E
:102610001F910F910895EF920F93CF93DF93D72FD0
:10262000C82FC9010E19009729F480E857FD05C08D
:1026300080E003C0BA010E94DA11602F681B7D2F71
:102640008C2FDF91CF910F91EF9008950F93CF933F
:10265000DF93D72FC82FC901009729F480E857FDD1
:1026600005C080E003C0BA010E94DA11602F680F34
:102670007D2F8C2FDF91CF910F910895EF920F93C3
:10268000972F23E0029FB0011124759567956E0D79
:10269000792F0F91EF900895E42FF0E0EE0FFF1FD8
:1026A000E351FE4F6081621B0895E42FF0E0EE0FCE
:1026B000FF1FE451FE4F6081621B0895622F089551
:1026C000E82F86FDE0952E2F2F7086FD2F5FE69573
:1026D000E695E695E670F0E0E159FE4F9181929F14
:1026E000902D212D112492959F702295207F922B61
:1026F0002081920F87FD919580E8890F0895AC01A4
:102700008230910508F408959FEF413E8EE158070D
:1027100040F49A0195E0369527959A95E1F798E06F
:10272000920F61E0E62FE90FFF27FF1F9F0135950C
:102730002795822F229FF001239FF00DF00D112489
:102740004E175F0738F49FEF920F961758F78FEFE9
:10275000860F08952F3FE9F361E0620FF6CF0F93E4
:10276000CF93DF93D72FC82F47FD419588E390E0A3
:10277000841B910947FD9395889FB001899F700D37
:10278000700D1124229FC001239F900D900D1124E4
:10279000860F971F0E947F13982F990F890F682F1C
:1027A000600F7D2F8C2FDF91CF910F91089530E036
:1027B00020E0869F212D969F200D311D1124C901F7
:1027C0000895AF92BF92CF92DF92FF920F931F9323
:1027D000CF93DF93362F472FE82FF0E0E752FB4EE1
:1027E00071110FC0E4918E2F2E2F6E2F722FDF915B
:1027F000CF911F910F91FF90DF90CF90BF90AF903E
:102800000895C72FD0E02491F22E022F10E056E059
:10281000659FC0011124EFEFF0E0BF010E94D533A6
:10282000832F90E0880F991F35E5369FD001379FA1
:10283000B00D11248A1B9B0B982F990F980F6F01D5
:10284000CC1ADD0AC09ED001C19EB00DD09EB00D45
:1028500011248B2F499FA0011124452F55276F016B
:10286000C41AD50AC09EA001C19E500DD09E500D25
:1028700011245F01A91AB108AC9E6001AD9ED00C75
:10288000BC9ED00C1124CD2CDD24EC19FD09E09F59
:10289000E001E19FD00DF09FD00D1124ED2F6230AB
:1028A0007105A1F050F46115710509F49ECF6130F6
:1028B000710581F0EB2F852F98CF6430710569F099
:1028C00080F06630710509F490CFF4CFE22F2B2F02
:1028D0008D2F8BCFE22F252F88CFEB2F822F2D2FFF
:1028E00084CF2B2F8F2DE52F80CF9F92AF92BF9259
:1028F000CF92DF92EF92FF920F931F93CF93DF93CC
:102900006C01C091180184E1C89FC02D112414E10D
:102910001C0FB12E153610F034E6B32E6091E10590
:10292000669566958091D5059091D6050E94D7133E
:10293000F82E80E48F0D0E94601390E8A92EA80E57
:102940008F2D0E94601320E8922E980ED0E0CB15B8
:1029500080F081E0143608F080E0DF91CF911F9184
:102960000F91FF90EF90DF90CF90BF90AF909F902E
:102970000895FE01EC54FD4F808190911901892347
:10298000A1F06091DE057091DF058091E005EF2CEC
:102990000C2F292D4A2DF60109950E94E113462F8F
:1029A000282F672FCE010E9477122196D0CF7F92D9
:1029B0008F929F92AF92BF92CF92DF92EF92FF924F
:1029C0000F931F93CF93DF935C01C091180184E1B3
:1029D000C89FC02D112414E11C0FF12E153610F0E4
:1029E00034E6F32E6091E10566958091D5059091CE
:1029F000D6050E94D713782ED0E0CF1590F081E055
:102A0000143608F080E0DF91CF911F910F91FF9075
:102A1000EF90DF90CF90BF90AF909F908F907F907E
:102A20000895FE01EC54FD4F808190911901892396
:102A3000C9F1CE01880F991F8A579E4FFC01EA59B0
:102A4000FF4F2081422F4057550B6A0189599F4FF4
:102A5000FC018081282F2052330B4901449F9001B3
:102A6000459F300D300D1124889CC001899C900D2C
:102A7000900D1124820F931F0E947F13082F6091E5
:102A8000DE057091DF058091E005E72C9401A60139
:102A9000F50109950E94E113462F282F672FCE01DB
:102AA0000E9477122196A9CFCF92DF92EF92FF92E8
:102AB0000F931F93CF93DF937C01C091180184E1A2
:102AC000C89FC02D112414E11C0FD12E153610F013
:102AD00034E6D32E6091E10566958091D5059091FD
:102AE000D6050E94D713C82ED0E0CD1568F081E03E
:102AF000143608F080E0DF91CF911F910F91FF9085
:102B0000EF90DF90CF900895FE01EC54FD4F80814F
:102B100090911901892311F1CE01880F991F8A57CD
:102B20009E4FFC01E959FF4F20812052330B8A59F7
:102B30009F4FFC0140814057550B6091DE0570911D
:102B4000DF058091E0050C2DF70109950E94E11346
:102B5000462F282F672FCE010E9477122196C5CFCE
:102B6000DF92EF92FF920F931F93CF93DF937C013D
:102B7000C091180184E1C89FC02D112414E11C0FDD
:102B8000012F153608F004E66091E105669566951B
:102B900021E0620F08F46FEF8091D5059091D60582
:102BA0000E94D713D82ED0E0C01760F081E0143611
:102BB00008F080E0DF91CF911F910F91FF90EF908F
:102BC000DF900895FE01EC54FD4F80819091190132
:102BD000892391F06091DE057091DF058091E00519
:102BE0002D2D4C2FF70109950E94E113462F282F18
:102BF000672FCE010E9477122196D6CF80E00895EC
:102C0000F894E82FE295EF70F0E031A1282F2F70B3
:102C100081E090E001C0880F2A95EAF7982F9095FF
:102C2000932391A392A1892B82A3789408959091E4
:102C3000A10592FF06C0282F28712830F9F4877F5C
:102C4000846093FF06C0282F28712831F1F4877E15
:102C500084612091A20520FF06C0382F38713830DA
:102C6000D9F4877F816021FF06C0282F2871283181
:102C7000D1F4877E816194FD877E0895282F247189
:102C80002430F9F68B7F8860DCCF282F2471243123
:102C900001F78B7E8861DDCF382F3171313019F724
:102CA0008E7F8860E0CF282F2171213121F78E7E21
:102CB0008861E1CFCF93DF93EC018238910581F1F8
:102CC000B0F58133910509F491C020F58932910561
:102CD00009F485C08A9709F490C0C11521E5D2078F
:102CE00008F0AAC0C11530E5D30708F0F2C0CF3B09
:102CF000D10508F089C0C83AD10508F0DFC0C53A4F
:102D0000D10508F0D3C0C430D105F8F4C130D105E5
:102D1000E1F040C08533910509F45AC0C997E9F63E
:102D20008091A105837089F0C0EED0E00EC0833E93
:102D3000910599F170F4803E910501F1823E910573
:102D400061F68091A10582FD21C0CE01DF91CF9176
:102D50000895863E910561F1873E910571F1843EAB
:102D6000910509F0BACF8091A20581FFEECF809145
:102D7000A105C7EED0E084FD0DC0E7CF8091A1058D
:102D800080FDF7C09091A20590FFDFCFC3EED0E0A9
:102D900084FFDBCFD0E0C0E0D8CF8091A10582FDD9
:102DA000EBC09091A20590FDBFCF84FFCECFF2CFB4
:102DB0008091A10583FDDDCFC8CF8091A10583FD62
:102DC000DEC09091A20591FFF0CFC4EED0E0BDCF60
:102DD0008091A10585FFB9CFC9E2D0E0B6CF80913F
:102DE000A10585FFB2CFC5E3D0E0AFCF8091A105AB
:102DF00086FFABCFCAE2D0E0A8CF8091A10586FFC5
:102E0000A4CFC1E3D0E0A1CFC11540E2D40760F464
:102E1000C11581E0D80708F098CFCE01815E9109F5
:102E2000079708F492CFB6CFC11590E4D90708F4FC
:102E3000B1CFDF70D06A89CFC11524E5D20778F40D
:102E4000C11533E5D30708F072C0C11542E5D407B8
:102E500008F05CC0DC2FCC27C16FD06A76CFC115DB
:102E60008AE5D80778F4C11599E5D90708F073C049
:102E7000C11528E5D20708F48DCFDC2FCC27C06F11
:102E8000D06A63CFCE0190568115904208F082CF70
:102E90008D2F8F710E94171690E0982F8827882712
:102EA0009F719C012C2BE901D0624FCFC55AD0E015
:102EB000C15EDE4FC881D0E0D06447CFC85AD0E0B1
:102EC000CC0FDD1FCE5DDE4F0990D881C02DD464BC
:102ED0003CCFCE0164E0969587956A95E1F78370C3
:102EE0002C2F26952695237040E2249F90011124D3
:102EF000382B8C2F8370C1E0D0E002C0CC0FDD1FD7
:102F00008A95E2F7C22BD32BDC681FCFCE018370EA
:102F1000992721E030E002C0220F331F8A95E2F7A3
:102F2000C695C69580E2C89FE0011124EBCFCE0183
:102F30008370992721E030E002C0220F331F8A9569
:102F4000E2F7C695C69590E2C99FE0011124C22B15
:102F5000D32BDA68FACE8C2F8F700E94171634E0CC
:102F6000D695C7953A95E1F7CF709C2FEC01D069C3
:102F7000ECCEC9E3D0E0E9CEC2EED0E0E6CEC6EEBC
:102F8000D0E0E3CE80919E0390919D03892B909198
:102F90009C03892B80931A03E0919905F0919A057F
:102FA000309799F090911701992349F09091A105DC
:102FB00097FF05C080931B0386E080931A0302806D
:102FC000F381E02D8AE193E00994089580919B03B9
:102FD00090916A03981301C008958F5F8770FACFAC
:102FE00021E1929F800D1124982F977086958695E8
:102FF000869523E0829FF0011124E35CFC4F50E0B2
:1030000040E080E0219130E0092E02C036952795FE
:103010000A94E2F721703327042E01C0220F0A948C
:10302000EAF7822B4F5F5F4F4330510559F7089500
:1030300021E1929F800D1124982F977041E001C0EB
:10304000440F9A95EAF786958695869593E0899F31
:10305000F0011124E35CFC4F90E080E070E05191BE
:10306000DF0111979B01082E02C0369527950A941F
:10307000E2F7217021952527242325272C930196FB
:103080008330910561F7089590E080E00E948611F9
:1030900090E080E00E94701110929D0310929C03BA
:1030A0000C94C2178093E3050C9444188091E305B7
:1030B000982F9670963019F488600C945218877F78
:1030C000FCCF21E030E001C0220F8A95EAF720957D
:1030D0008091E30582230C94521821E030E001C076
:1030E000220F8A95EAF78091E305822B0C945218FF
:1030F00080939F030C944418882341F0809590910D
:103100009E03892380939E030C94C21708958823FD
:1031100039F090919E03982B90939E030C94C217C4
:103120000895882379F19CEF980F913A38F4682F2D
:103130008AE193E00E9411110C94C21790E2980F5B
:10314000983088F4877021E030E0A90102C0440F74
:10315000551F8A95E2F7CA01809590919E038923B5
:1031600080939E03E9CF9BE5980F933020F490E085
:1031700080E00C948611885A873120F490E080E03A
:103180000C9470110895CF93C82F882309F467C059
:103190008CEF8C0F813AC0F580911701882311F1D3
:1031A0008091A10587FF1EC0EC2FE695E695E69578
:1031B000F0E0E65EFC4F828190E04C2F477021E00A
:1031C00030E002C0220F331F4A95E2F78223932397
:1031D000892B91F06C2F8AE193E00E9411110E94DB
:1031E000C2170AC0ECE1F3E082E293E02191C2173A
:1031F00089F38E179F07D1F76C2F8AE193E00E9425
:103200003B11CF910C94C21780E28C0F883068F488
:10321000C77021E030E001C0220FCA95EAF7809123
:103220009E03822B80939E03ECCFEBE5EC0FE33003
:1032300040F4F0E0E15EFE4F808190E0CF910C948D
:103240008611C85AC73158F4EC2FF0E0EE0FFF1F7B
:10325000EE5DFE4F80819181CF910C947011CF91E2
:103260000895809108048B30F0F480913B0390E046
:10327000019665E070E00E94F53380933B0324E003
:1032800030E0281B390B4DE052E0249FC001259F00
:10329000900D349F900D11248E55984F0C94EB0E89
:1032A00085E995E0FBCF8431D8F380913A0390E033
:1032B00001968170992780933A0321E030E0281B22
:1032C000390B4DE052E0249FC001259F900D349FA3
:1032D000900D112485589E4FE1CFCF92DF92EF924F
:1032E000FF920F931F93CF93DF936C017B0164E6F2
:1032F00070E088E70E94D432EC0197FD12C010E024
:1033000000E0F601E00FF11F849164E670E00E9496
:103310004E33EC01892B29F40F5F1F4F0E151F054B
:1033200081F70E94D133CE01DF91CF911F910F9190
:10333000FF90EF90DF90CF90089580919505909148
:103340009605911103C091E089270895882369F0BB
:1033500062E070E08BED95E10E946D19892B19F008
:103360008091950508951092950580919505EBCF74
:10337000CF93C0919505809196058823D1F00E9446
:103380000511605A75418F4F9F4F6093910570935F
:1033900092058093930590939405C11108C062E053
:1033A00070E089ED95E10E946D19892B29F0C0919B
:1033B00095058C2FCF91089581E080939505F7CFE7
:1033C00010929E0380911701ECE1F3E0882359F0FD
:1033D0008091A10587FF07C08EE1DF011D928A95CC
:1033E000E9F70C94441886E0F8CF1F93CF93DF934E
:1033F000CDB7DEB7AA970FB6F894DEBF0FBECDBF2C
:103400008DEC95E02091F100DC012D93CD01B5E02C
:10341000853D9B07B9F78091CE05833009F472C0D2
:10342000B8F4813009F449C0823009F4B3C0809106
:10343000E80083FF8BC28091CD059091CE059A3034
:1034400008F084C2E92FF0E0ED55F94C0C944A34B1
:103450008A3009F48EC08B3009F471C0893039F795
:103460008091CD05813219F78091D1059091D205D7
:10347000009711F00297D9F68091E800877F80933A
:10348000E8008091E80082FF38C09091F3008091BD
:10349000F200029731F48091F100813011F0863012
:1034A00021F48091F1008093A8058091E8008B774A
:1034B0008093E8000E94D40FBACF8091CD05813A65
:1034C00009F0B5CF8091E800877F8093E800809174
:1034D000D1059091D205892B61F460E289EA95E0EB
:1034E00070E00E9486108091E8008B778093E8005E
:1034F0009ECF60E090E080E0F3CF8091CB0581111A
:10350000C0CF95CF8091CD05813A09F090CF8091C1
:10351000D1059091D205892B09F089CF8091E800DF
:10352000877F8093E8008091E80080FFFCCF809146
:1035300017018093F1008091E8008E77B9CF8091D8
:10354000CD05813209F073CF8091D1059091D205DC
:10355000892B09F06CCF8091E800877F8093E80089
:103560000E94D40F8091CF05809317010E94E0192B
:103570005ECF8091CD05813209F059CF8091E8006E
:10358000877F8093E8000E94D40F8091D0058093BC
:10359000A7054DCF8091CD05813A09F048CF8091A4
:1035A000E800877F8093E8008091E80080FFFCCFEF
:1035B0008091A705BECF803899F0823809F0C6C146
:1035C0008091D1058F70873008F0C0C18093E900E9
:1035D0008091EB0085FB882780F91092E90006C0F6
:1035E0008091C9059091CA05911182609091E8007F
:1035F000977F9093E8008093F1001092F100809102
:10360000E8008E779FC1882309F48DC1823009F0CC
:103610009DC18091CF05811190C18091D1058F709E
:103620002FEF280F263008F091C18093E9002091F8
:10363000EB0020FF82C1933031F48091EB00806277
:103640008093EB007AC19091EB0090619093EB0036
:1036500021E030E001C0220F8A95EAF72093EA00CA
:103660001092EA008091EB008860EACF81116EC170
:103670001091CF051F778091E3008078812B809394
:10368000E3008091E800877F8093E8000E94D40FD8
:103690008091E80080FFFCCF8091E30080688093F8
:1036A000E30082E0111183E08093CB054FC1805885
:1036B000823008F04BC12091CF053091D0052C3DD0
:1036C000E3E03E07A1F583E08A838AE289834FB76E
:1036D000F894DE01139620E03EE051E2E32FF0E0A3
:1036E00050935700E49120FF03C0E295EF703F5FD5
:1036F000EF708E2F90E0EA30C0F0C7968D939D93C7
:103700002F5F243159F74FBF8091E800877F809366
:10371000E8006AE270E0CE0101960E948610809176
:10372000E8008B778093E80011C1C096E7CF8091C5
:10373000D1059091D205432F55274330510509F407
:103740004AC078F54130510509F47AC08BE590E024
:10375000E5E7F7E14230510509F0F8C02091E800B3
:10376000277F2093E8002091D3053091D40582175C
:10377000930708F49C0140E02115310509F065C06C
:10378000411163C08091E80082FDC9CF8091CB05D3
:10379000882329F2853019F28091E80083FFF2CF67
:1037A000BECF4132510509F43CC04232510509F007
:1037B000CDC08330910508F0C9C0FC01EE0FFF1F9A
:1037C000E658FE4F0190F081E02D89589E4FDC01B4
:1037D0008C9190E01AC0332721303105D1F02115AA
:1037E000310561F02230310509F0B0C0E2EEF7E1B9
:1037F000E4918E2F90E0E2EEF7E107C0E0E0F8E11F
:10380000E4918E2F90E0E0E0F8E1009709F49EC08B
:10381000A5CFEEEEF7E1E4918E2F90E0EEEEF7E12A
:10382000F4CF8330910508F091C0880F991FFC01F7
:10383000E058FE4F0190F081E02D89E090E08ECFBE
:1038400082E190E0E0EDF7E189CF8091CB0588231C
:1038500009F465CF853009F462CF8091E80083FDDB
:103860005ECF8091E80082FD8DCF8091E80080FFDF
:1038700083CF9091F3008091F2002115310519F06A
:103880008830910550F041E0089709F040E08091C0
:10389000E8008E778093E8006FCF44914093F10069
:1038A0003196215031090196E8CF803809F04EC099
:1038B0008091E800877F8093E8008091CC05809319
:1038C000F1009DCE811142C01091CF051230F0F56C
:1038D0008091E800877F8093E8001093CC050E94D8
:1038E000D40F112311F084E005C08091E30087FD1F
:1038F000FACF81E08093CB0542E061EC81E00E9449
:10390000F30F42E261EC84E00E94F30F42E261ECCB
:1039100082E00E94F30F42E260EC83E00E94F30F2A
:103920008091CB0513C08091CF05813079F481E07F
:10393000933009F080E08093CA051092E9008091ED
:10394000E800877F8093E8000E94D40F8091E80010
:1039500083FF0AC08091E800877F8093E800809110
:10396000EB0080628093EB00AA960FB6F894DEBF5E
:103970000FBECDBFDF91CF911F910895CF93DF93FD
:10398000C091ED07D091EE078A30C1F42091E40593
:10399000CE018D5E9540622F70E00E94D533281BCA
:1039A000822F66E00E94E933C82FC15018F4DF91DE
:1039B000CF91089580E20E94BE1CF7CF8D30E9F4CC
:1039C000CD5ED5402091E405622F70E0CE010E94CB
:1039D000D533281B822F9E01280F311D211532401F
:1039E00018F080E0D0E0C0E0C80FD11DC351DA4F1D
:1039F000D093EE07C093ED07DACF96E0FE01A5EE77
:103A0000B5E001900D929A95E1F7803E08F458C018
:103A100086E0FE0111928A95E9F7C091ED07D091F9
:103A2000EE0746E050E0BE0185EE95E00E9482344C
:103A30009E012D5E3540892B41F1C90145E09695E7
:103A400087954A95E1F741E050E0BA0102C0660F60
:103A5000771F8A95E2F7CB016091EB057091EC0539
:103A6000862B972BB9016B5F7F4FE5E076956795C5
:103A7000EA95E1F702C0440F551F6A95E2F7842BDF
:103A8000952B9093EC058093EB052A5F3F4F409177
:103A9000E405642F70E0C9010E94D533481B46300D
:103AA00010F4240F311D211572E0370710F030E0BB
:103AB00020E023513A4F3093EE072093ED0777CF64
:103AC000F6E08F9FB00111246C5F774E46E050E026
:103AD000CE010E947934A1CFCF93DF93EC01FE0198
:103AE0008491811103C0DF91CF9108950E94BE1C83
:103AF0002196F5CF8093A3057093A5056093A40547
:103B00008091CB058430F9F48093E9008FEF909198
:103B1000E800815095FD06C095ED9A95F1F70000FB
:103B20008111F5CF8091E80085FF0DC050E040E0A5
:103B300063E070E083EA95E00E94AA0F8091E800BC
:103B40008E778093E8000895BC0184E00C947A1D80
:103B5000BC0183E00C947A1DCF93DF93EC0180913C
:103B600017018823B1F18091A10587FF32C060E27F
:103B700084E08093E9008FEF9091E800815095FDFB
:103B800006C095ED9A95F1F700008111F5CF80916F
:103B9000E80085FF1BC08091170170E050E040E015
:103BA000811104C050E040E068E070E0CE010E9466
:103BB000AA0F8091E8008E778093E80080E2FE01F2
:103BC000A9EAB5E001900D928A95E1F7DF91CF91D6
:103BD000089568E081E0CDCF81E08093E00080E24D
:103BE0008093D8001092C9008FE19EE40197F1F70D
:103BF00000C0000087E090EBDC018093EF0790931A
:103C0000F007A093F107B093F20788E19CE00FB6AC
:103C1000F894A895809360000FBE90936000FFCF4A
:103C20006A9A3EB13B7F2EB124604FB7F89485E687
:103C300094E0FC015191CF0168E02EB9000000C072
:103C400057FF3EB9550F000000C000C000C03EB98C
:103C500000C06A9591F7F5E081399F0751F74FBF92
:103C60008FE594E00197F1F700C0000008951F93DD
:103C7000CF93DF93182FD0E0C0E0893311F4C0E573
:103C8000D0E0812F0E94C318209731F4812FDF915B
:103C9000CF911F910C9491188FE99FE00197F1F754
:103CA00000C000002197F0CFCF93DF93CFEBD1E09E
:103CB00060E0CE010E94BD342196C11584E0D80792
:103CC000B9F7DF91CF9108956F927F928F929F9273
:103CD000AF92BF92CF92DF92EF92FF920F931F931A
:103CE000CF93DF938DEDC82E85E1D82E95E1E92E97
:103CF000FF24F394E701CC5CD10936011BC0F50128
:103D000085909490692DC8010E94BD34682DC8012A
:103D100001960E94BD3482E0A80EB11C0E5F1F4FB9
:103D2000C017D10761F782E2680E711CA296CE150A
:103D3000DF0529F08E01025211095301E0CF7E0107
:103D40008CECE80EF11C8CECC80ED11C8DEAE81648
:103D500082E0F80679F6DF91CF911F910F91FF90E5
:103D6000EF90DF90CF90BF90AF909F908F907F901B
:103D70006F900895CF93C82F6FEF811161E283E2B6
:103D800090E00E94BD346FEFC11162E184E290E0E7
:103D90000E94BD346FEFC11160E185E290E0CF91E8
:103DA0000C94BD3480E00E94BA1E60E086E290E090
:103DB0000E94BD340E94641E0E94541E81E00C9437
:103DC000BA1E0F931F93CF93DF93C42FD0E0CC0F75
:103DD000DD1F22E2629FC00DD11D11243CEC839FA8
:103DE000C00DD11D1124CE0187960E949F34082F4B
:103DF00010E0102F0027CE0188960E949F34980172
:103E0000282BC901DF91CF911F910F910895462F63
:103E1000823038F4763028F4613118F4672F0C942E
:103E2000E11E90E080E00895CF92DF92FF920F9321
:103E30001F93CF93DF936C010091E30580919F0363
:103E4000082BC7E0D0E010E0FC2EC8010C2E02C009
:103E5000959587950A94E2F780FD0CC02197A0F70D
:103E6000F12C8F2DDF91CF911F910F91FF90DF905B
:103E7000CF900895B6018C2F0E94071F0E945A16FA
:103E8000019761F3EECFCF93DF93EC010E94141FF3
:103E9000BE010E94071FDF91CF910C945A16FC01BE
:103EA000808191810E94431F292F2F7092959F70CE
:103EB00092509E3078F4E92FF0E0E355F94C0C94E1
:103EC0004A34803F19F020F4883E20F481E00895C0
:103ED000843FE1F380E00895883EC0F3813FD1F74D
:103EE000F5CF822F869586958695089583E290E09A
:103EF0000E949F34813289F484E290E00E949F34D2
:103F0000823159F485E290E00E949F3491E0803143
:103F100009F090E0892F8170089580E0FCCFCF9365
:103F200084E090E00E949F34C82F82E290E00E94DB
:103F30009F34982F8C2FCF910895EDEDF5E08DE013
:103F4000808380911C0190911D01A0911E018183AD
:103F50009283A3838FE784838FEF858346E050E0CD
:103F60006CE170E0CF010E94AD341092DC05089541
:103F700090E080E00E94A734893E9E4F11F40C949B
:103F8000761F80E0089569EE7EEF90E080E00E9469
:103F9000DB3460E082E090E00E94BD3460E083E0CA
:103FA00090E00E94BD3410929F0360E084E090E0B6
:103FB0000E94BD3460E082E290E00E94BD3460E087
:103FC00085E090E00E94BD3460E086E090E00E94D1
:103FD000BD346FEF87E090E00E94BD3440E050E0D8
:103FE000BA0188E090E00E94CF3460E08DE090E07C
:103FF0000E94BD3440E050E0BA0188E190E00E94A8
:10400000CF3460E087E190E00E94BD3440E050E0B2
:10401000BA018CE190E00E94CF3470E060E080E271
:1040200090E00E94DB3440E050E0BA0188E190E08B
:104030000E94CF3480E00E94BA1E0E94D21E40E04F
:1040400050E0BA018FE090E00E94CF3440E050E0B1
:10405000BA0183E190E00C94CF341F920F920FB617
:104060000F9211242F933F934F935F936F937F93FE
:104070008F939F93AF93BF93CF93DF93EF93FF9370
:10408000D091E900DF708091EC00C82FC17080FDF5
:10409000C0E81092E9008091F000877F8093F000E3
:1040A00078940E94F5191092E9008091F0008860E0
:1040B0008093F000CD2BCF70C093E900FF91EF917A
:1040C000DF91CF91BF91AF919F918F917F916F9130
:1040D0005F914F913F912F910F900FBE0F901F90C6
:1040E00018951F920F920FB60F9211242F933F93A2
:1040F0004F935F936F937F938F939F93AF93BF93F0
:10410000EF93FF938091E10082FF09C08091E2006C
:1041100082FF05C08091E1008B7F8093E100809158
:10412000DA0080FF24C08091D80080FF20C08091F9
:10413000DA008E7F8093DA008091D90080FFA1C0E1
:1041400080E189BD82E189BD09B400FEFDCF81E037
:104150008093CB058091A605811109C00E945A0F5A
:104160000E9425108091E20084608093E20080919B
:10417000E10080FF17C08091E20080FF13C08091B2
:10418000E2008E7F8093E2008091E2008061809364
:10419000E2008091D80080628093D80019BC85E04D
:1041A0008093CB058091E10084FF2FC08091E200D5
:1041B00084FF2BC080E189BD82E189BD89B5982F3C
:1041C000917080FFFBCF8091D8008F7D8093D800C5
:1041D0008091E1008F7E8093E1008091E2008F7EEC
:1041E0008093E2008091E20081608093E200809100
:1041F000CC05882309F44BC084E08093CB050E9452
:10420000E0190E949C118091CB058091E10083FF11
:1042100027C08091E20083FF23C08091E100877F67
:104220008093E10082E08093CB051092CC058091D1
:10423000E1008E7F8093E1008091E2008E7F809389
:10424000E2008091E20080618093E20042E060E061
:1042500080E00E94F30F8091F00088608093F0006E
:10426000FF91EF91BF91AF919F918F917F916F914E
:104270005F914F913F912F910F900FBE0F901F9024
:10428000189519BC1092CB051092A60570CF80919D
:10429000E30087FD93E09093CB05B1CF78941F9214
:1042A0001FB61F9211248F939F93AF93BF9380915A
:1042B0009D0590919E05A0919F05B091A005019646
:1042C000A11DB11D80939D0590939E05A0939F0510
:1042D000B093A005BF91AF919F918F911F901FBE8A
:1042E0001F9018959C014FB7F89480919D0590916F
:1042F0009E05A0919F05B091A0054FBF821B930B17
:1043000008952FB7F89480919D0590919E05A091F6
:104310009F05B091A0052FBF08950F931F93CF93D2
:10432000DF93C62FD42F022FFC0182818823A1F0B6
:104330006093DB050E9481219093DA058093D90573
:10434000C77081E001C0880FCA95EAF7DF91CF916D
:104350001F910F910C9487188091DB05681335C06D
:104360008091D9059091DA050E947221883C9105CF
:1043700060F510E21D0FCD17B9F080E28C0F883088
:1043800040F4C77081E001C0880FCA95EAF70E9427
:104390007C18183048F481E09D2F977001C0880F79
:1043A0009A95EAF70E948718802F0E94371E1830CE
:1043B00098F4D77081E001C0880FDA95EAF7DF91B1
:1043C000CF911F910F910C947C18C77081E001C0B0
:1043D000880FCA95EAF7F3CFDF91CF911F910F9124
:1043E00008955F926F927F928F929F92AF92BF9249
:1043F000CF92DF92EF92FF920F931F93CF93DF93B1
:1044000000D000D00F92CDB7DEB77C01FC018381D4
:104410009481892B31F08081918189238F3F09F02C
:104420002FC50F900F900F900F900F90DF91CF91AD
:104430001F910F91FF90EF90DF90CF90BF90AF90C2
:104440009F908F907F906F905F9008950E94141FAF
:10445000182F682F89819A810E94181869817A81A2
:10446000812F0E94071F8C01F7012281222309F46A
:10447000FDC490568115F0E29F0750F0905E8115C3
:1044800030E1930728F0915C81159F4108F05AC0F4
:10449000C8019927AC01445051094432510518F024
:1044A0008B970E9740F4E091A903F0E0E255FC4FA2
:1044B00080818F5F8083C80182519F45409708F0BB
:1044C0009BC48FEF93E00E949F3402519FEBA92E73
:1044D000BB24B3948111A5CF01113DC01C821B8266
:1044E000662463948AE0582E85010F5F1F4FC50133
:1044F0000E949F3489831A82882309F492CF9FEF08
:10450000980F9330B8F58A83698292E0A90EB11CA6
:10451000C8010E949F348B83882309F482CF8E01C7
:104520000F5F1F4FF80120812223F1F2213009F0A3
:104530005BC0918182819130F9F40E5F1F4F0E9420
:10454000371E20C090E080E00F3F110511F008F009
:10455000A1CFC8019FCFA11454E0B50609F461CFE3
:10456000C5010E949F34811101C001508FEFA81A2C
:10457000B80AB2CF5801D3CF923039F40E5F1F4F33
:104580000E94C3180F5F1F4FCDCF933029F40E5FE9
:104590001F4F0E949118F6CF943019F00F5F1F4FF4
:1045A000F1CF0E5F1F4F30E020E0B8016F5F7F4F0B
:1045B000F80141818053990B8A30910550F02150C8
:1045C000310900F38FE99FE00197F1F700C0000087
:1045D000F6CF529EF001539EF00D11249C012E0F38
:1045E0003F1F842F8B01E1CFE22FF0E0ED5EFD4E07
:1045F0007490822F86958695869590E0FC01ED5FFC
:10460000FD4EE4902770F12C022E02C0F594E79441
:104610000A94E2F7E1E0EE22FF24FC01ED50FE4EA9
:10462000C490D12C022E02C0D594C7940A94E2F70C
:10463000F1E0CF22DD24FC01ED51FE4E8490912C5F
:1046400002C0959487942A95E2F721E0822299246A
:10465000E114F10419F081EE0E94C318C114D104D1
:1046600019F086EE0E94C318872D0E94371ECD28B0
:1046700019F086EE0E949118EF2819F081EE0E9441
:104680009118892809F47ECF8CE259CF81E00E94ED
:104690006D1803C081E00E9461180F900F900F9079
:1046A0000F900F90DF91CF911F910F91FF90EF909E
:1046B000DF90CF90BF90AF909F908F907F906F9042
:1046C0005F900C945618222309F4D8C382E0DFCF00
:1046D000053FECE51E0709F46EC008F468C0063F0C
:1046E0003CE5130709F46BC0222309F4DAC31092E6
:1046F000DB0503304DE5140708F068C00A3F5CE5B0
:10470000150730F4C80182509C45449708F063C0F7
:104710000E948F1F9093A2058093A10500319CE514
:10472000190709F440C108F0B8C00830FCE51F07BC
:1047300009F427C108F08CC004303CE5130709F4E4
:1047400012C108F072C002305CE5150709F401C11E
:1047500003301C4509F403C16091A1051091A20525
:1047600084E090E00E94BD34612F82E290E00E94DC
:10477000BD340F900F900F900F900F90DF91CF915D
:104780001F910F91FF90EF90DF90CF90BF90AF906F
:104790009F908F907F906F905F900C94E01927E22C
:1047A00045EE65EE4CC326E241EE60EE48C327E2DB
:1047B00045EE64EE44C326E241EE62EE40C327E2DA
:1047C00045EE66EE3CC328E241E0EBCF01368DE5D5
:1047D000180709F49DCF80919E0306319CE51907C7
:1047E00009F06CC38A7A91E009F490E090933C035D
:1047F00069E2811165E38AE193E00E943B110F9029
:104800000F900F900F900F90DF91CF911F910F910C
:10481000FF90EF90DF90CF90BF90AF909F908F90E0
:104820007F906F905F900C94C2178091A10580617A
:1048300006309CE5190709F48FC08091A1058860B6
:1048400007301C4508F488C08091A105806284C0AF
:104850008091A1058D7F0C30FCE51F0709F47CC019
:1048600070F48091A1058C600A303CE5130709F4CF
:1048700073C008F48AC08091A1058E7F6DC08091BD
:10488000A105877F0E305CE5150709F465C008F4C3
:1048900082C08091A1058F7E5FC00C3F9CE5190707
:1048A00009F47DC068F50431FCE51F0709F48FC0E9
:1048B00080F402313CE5130709F479C08091A10529
:1048C0008F7B03311C4508F447C08091A105837F8D
:1048D00043C00A3F5CE5150709F449C008F04DC024
:1048E00005311C4509F038CF8091A10582FB99273D
:1048F00090F921E0922790FB82F990FB83F92CC07C
:104900000115EDE51E0709F458C088F48091A20551
:1049100083600E3F2CE5120769F18091A2058D7F1F
:104920000F3F1C4538F18091A2058C7F23C00230D7
:104930004DE5140709F45AC008F452C001361D456C
:1049400009F00ACF9091A105892F8F7E94FF806195
:1049500003C08091A10581608093A105FDCE809167
:10496000A1058260F9CF8091A1058460F5CF809187
:10497000A20581608093A205EFCE8091A20582609E
:10498000F9CF8091A1058064E7CF0E94E019809162
:10499000A1058068E1CF8091A1058B7FDDCF80915B
:1049A000A2058E7FE7CF8091A1058F7DD5CF0E9494
:1049B000E0198091A1058F77CFCF8091A205982F24
:1049C000909591708E7F892B90FB81F9D3CF0E94B7
:1049D000E0199091A105892F97FB87F98058BCCFEA
:1049E00061E08EE090E00E94BD34B6CE60E0F9CF89
:1049F0008091DD0591E089278093DD0510921B01F0
:104A00008091DC0581608093DC050BCD42E652E1AC
:104A10006BE672E10F900F900F900F900F90DF9167
:104A2000CF911F910F91FF90EF90DF90CF90BF90AB
:104A3000AF909F908F907F906F905F900C94BF117C
:104A40004BE652E162E672E1E5CF40E552E169E50D
:104A500072E1E0CF49E552E160E572E1DBCF48E386
:104A600052E164E472E1D6CF44E452E168E372E1DA
:104A7000D1CF4CE252E160E272E1CCCF44E052E1AE
:104A800062E172E1C7CF42E152E164E072E1C2CF7C
:104A900081E00F900F900F900F900F90DF91CF91CA
:104AA0001F910F91FF90EF90DF90CF90BF90AF904C
:104AB0009F908F907F906F905F900C942E0F83E06B
:104AC000E8CF0E94E0192FEF34E34CE02150304052
:104AD0004040E1F700C000000E94EC1D0F900F90D5
:104AE0000F900F900F90DF91CF911F910F91FF903A
:104AF000EF90DF90CF90BF90AF909F908F907F907E
:104B00006F905F900C94C31F0E94F017D82E07C2BD
:104B1000092F0F70907F11F00295007F812F2223C3
:104B2000C9F0002369F090E2910F983010F0111154
:104B30000BC080919E03082B00939E030E94C21716
:104B4000812F0E94C31817C080919D03082B0093EA
:104B50009D03F4CF0E949118002369F00095105E28
:104B6000183010F0B11025C080919E0308230093E7
:104B70009E030E94C21758E0C51AD10884E0C816E7
:104B8000D10408F04ECC0F900F900F900F900F9023
:104B9000DF91CF911F910F91FF90EF90DF90CF9019
:104BA000BF90AF909F908F907F906F905F900C948C
:104BB0009C1180919D03082300939D03DACF892FD8
:104BC0008F70907F903211F08295807FF1E0BF125C
:104BD0000CC0222329F0363070F60E948718CBCF04
:104BE000353048F60E947C18C6CF222341F033238B
:104BF000A1F340FFA5CF4F70F7014583EECF3323DC
:104C000089F3193349F4FFEF27EE33E0F1502040E8
:104C10003040E1F700C00000812F0E949118ABCF17
:104C2000892F86958695837061F0813009F0A3CF36
:104C3000812F9370211102C090E080E00E947011DA
:104C40009ACF812F9370211102C090E080E00E94E2
:104C5000861191CF892F8370A1F521118CCF812FDF
:104C6000829586958770880F880F412F4F70082E88
:104C700001C0440F0A94EAF7212F207114FF07C0E6
:104C80002FE030E001C0220F8A95EAF72095969533
:104C900096959370923081F0822F842B933030F46C
:104CA00080919F03913029F0242B82230E94781851
:104CB00062CF842B822BFACF242B80919F038227F3
:104CC000F5CF8695222311F0892F8170882309F46E
:104CD00052CF812F829586958770880F880F412F3C
:104CE0004F70082E01C0440F0A94EAF7212F20715B
:104CF00014FF07C02FE030E001C0220F8A95EAF7C9
:104D00002095969596959370923081F0822F842B02
:104D1000933030F48091E305913029F0242B8223E5
:104D20000E94521828CF842B822BFACF242B8091FB
:104D3000E3058227F5CF092F0F70222329F0802F5A
:104D40000E946D18812F49CF812F0E947C18802FDF
:104D50000E94611810CF812F41EF141789F141177C
:104D600050F050EF1517B9F02223B1F13111E8CE10
:104D7000892F8F7129C0E2EF1E1749F1F3EF1F133E
:104D8000F3CF80E0222361F29F7181E001C0880FA0
:104D90009A95EAF7C5CF222379F0353008F0EBCEAB
:104DA000292F2F7181E090E001C0880F2A95EAF742
:104DB0009091E3058927B4CF363008F0DCCEF0CFF0
:104DC000892F8F71222321F20E946D18D4CE892F52
:104DD0008F712223C9F3BCCF332359F0893309F0F3
:104DE0001BCF2FEF37EE43E0215030404040E1F73A
:104DF00011CF892F8F71ACCF00319FE5190709F4CE
:104E000045CC0131EFE51E0709F45DCC033F3CE5DD
:104E1000130709F4C8CC08F05BCC083D5CE5150726
:104E200009F4BDCC093D8CE5180709F4CCCC073D4D
:104E30009CE5190709F058CC26E241EE61EEC70166
:104E40000F900F900F900F900F90DF91CF911F91C7
:104E50000F91FF90EF90DF90CF90BF90AF909F9019
:104E60008F907F906F905F900C948D218031FFE543
:104E70009F0709F40FCC81319F4541F682E00BCCAE
:104E800085E0DE01119601900D928A95E1F7F70118
:104E9000228189819A812111D9CA0E94F017182F85
:104EA000DDCA06311C4569F580913C0369E2811138
:104EB00065E38AE193E00E941111A1CC82720A3C61
:104EC0003CE5130709F4D5CD08F05AC0053C5CE574
:104ED000150709F4BACDF0F5033CECE51E0709F41B
:104EE00095CD08F0ADCD023C3CE5130709F480CD2B
:104EF0000115ECE51E0709F4E4CD0E3D1C4509F44F
:104F0000EDCDF70100811181C801222309F4FCCD08
:104F10000E94141FD82E682FC8010E941818B801CB
:104F20008D2D0E94071F0E945A16182FB82EF701C8
:104F300022814581342F32953F70892F82958F7061
:104F4000C82ED12C8C3008F016CEF601E554F94C61
:104F50000C944A34073C4CE5140709F480CD08F45E
:104F600079CD083C9CE5190709F47ECD40E252E179
:104F70006CE272E1093CECE51E0709F44BCDB8CFB9
:104F80000F3CFCE51F0709F49ACD90F40C3C4CE56E
:104F9000140709F478CD08F471CD0D3C8CE51807A1
:104FA00009F476CD0E3C9CE5190709F43ACAA0CF66
:104FB000063DECE51E0730F487E0013D1C4508F492
:104FC00068CD2FCA0D35100709F42BCA91CF1F9356
:104FD000CF93DF9380916903807FA9F4809166036A
:104FE000882389F080919B03D0916A0360916403C8
:104FF00070916503A0916703B0916803C62FC72322
:1050000016E0D81304C0DF91CF911F91089590E06E
:10501000109711F0CF3F19F401968770F2CF189FC7
:105020009001199F300D1124F901E559FC4F418180
:105030004713F2CF40814613EFCF42814111ECCFAD
:10504000438154814A1B5B0B483C510528F78091F2
:1050500069038F70806180936903F901E059FC4F07
:1050600080818F708061808384E693E00E94F121CB
:10507000DF91CF911F910C94E617AF92BF92CF9220
:10508000DF92EF92FF920F931F93CF93DF93CDB7F1
:10509000DEB761970FB6F894DEBF0FBECDBF8C01AF
:1050A00085E0F801DE011D9601900D928A95E1F7E9
:1050B000F801E28084E6A82E83E0B82E60916703B1
:1050C000709168036115710509F432C19091640310
:1050D00040916503892F84238F3F09F429C12081E2
:1050E0003181C380D480F0906603F601E61BF70B94
:1050F000FF2009F4E8C080916903582F507FE83CF5
:10510000F10508F0ABC0511177C0FE2C431321C04C
:1051100092131FC0E1101DC08F70806180936903DE
:10512000C5010E94F12180916903F80185838F2DCB
:1051300061960FB6F894DEBF0FBECDBFDF91CF9161
:105140001F910F91FF90EF90DF90CF90BF90AF90A5
:105150000895CD2829F0822F83238F3F09F003C1C2
:1051600080E0F82FF170DF2E80FF3CC080919B0320
:1051700040916A0356E0841315C02D873E878D85C4
:105180009E850E94431F292F22952F702230F0F018
:10519000243018F59F70F1F0F8019581907FD1F4DB
:1051A000D12C1EC090E0589FF001599FF00D1124A2
:1051B000E559FC4F6181361306C06081261303C098
:1051C0006281E6120FC001968770D5CF9F7011F0F3
:1051D000882331F3805E883018F3C8010E94F121E2
:1051E000FD2CA5CFEE2009F4A2CF80916903816048
:1051F00080936903F12C9BCF431306C0921304C024
:10520000F801EE2009F479C0C8010E944F1F8823DD
:1052100009F1EE20F9F080916903803270F020915D
:1052200064033091650338872F831986DB86CA862D
:105230008C87CE0107960E94F12186E0F801A4E652
:10524000B3E001900D928A95E1F70E94E727FF24D1
:10525000F3946DCFC8010E94F121F9CF51110AC01A
:1052600084E693E00E94F12186E0F50111928A958F
:10527000E9F7C0CF43130FC092130DC0E1100BC06C
:10528000F8018583C8010E94F12186E0F5011192A1
:105290008A95E9F74CCFC8010E944F1F8823D1F2AD
:1052A000EE20C1F280916903803238F220916403CC
:1052B000309165033A8329831B82DD82CC828E8301
:1052C000CE010196B8CFE83CF105F8F6FE2CEE20B1
:1052D00009F243131FC092131DC08091690380FD22
:1052E00010C0982F907F69F0F8018583903F31F0CE
:1052F000982F907F905F8F70892B8583C8010E94C3
:10530000F12186E0F801A4E6B3E001900D928A95C0
:10531000E1F70DCFC8010E944F1F81118ECF809100
:105320006903816080936903C8010E94F121FFCE67
:10533000EE2009F48FCFC8010E944F1FF82E88235A
:1053400009F488CF86E0F801A4E6B3E001900D925D
:105350008A95E1F780916403909165030E94431F51
:105360000E94E727E4CE81E08E25FBCE1F93CF93EA
:10537000DF93CDB7DEB767970FB6F894DEBF0FBEE9
:10538000CDBF4B8B5C8B6D8B7E8B8F8B61111092A5
:105390009D031A8A198A85E0FE017396DE011D9627
:1053A00001900D928A95E1F786E0FE013D96DE01BF
:1053B000179601900D928A95E1F7CE0107960E940B
:1053C0003D28882389F016E080919B0390916A0321
:1053D000891349C067960FB6F894DEBF0FBECDBFE4
:1053E000DF91CF911F91089586E0FE013796DE018F
:1053F000119601900D928A95E1F78A859B85892BFC
:1054000011F38F81988589238F3FE9F220916A03F8
:1054100030E0C90101968770992740919B03481796
:10542000190671F40E94E01910926A0310929B030E
:1054300086E0E4E6F3E0DF011D928A95E9F7C3CF49
:1054400096E0929FD001939FB00D1124A559BC4FB7
:10545000FE01319601900D929A95E1F780936A03CF
:105460000E94E617B0CF819FC001112485599C4F3F
:105470000E943D28882309F4ADCF80919B0390E0E2
:1054800001968770992780939B039ECF2F923F921E
:105490004F925F926F927F928F929F92AF92BF9244
:1054A000CF92DF92EF92FF920F931F93CF93DF93F0
:1054B000CDB7DEB768970FB6F894DEBF0FBECDBF8D
:1054C0008E010F5F1F4F88E1F80111928A95E9F76D
:1054D00020E5E22E21E0F22E680136E5232E31E0B0
:1054E000332EAA24A394B12C57E6852E51E0952E95
:1054F000F70181917F018F3F09F44FC0F894E82FA5
:10550000E295EF70F0E021A18F70A50102C0440F79
:10551000551F8A95E2F7CA01922F982B91A392A169
:105520008095892382A3789400C0E6E5F1E041E00C
:1055300050E060E070E0412C512C320121912F3F6E
:1055400009F46DC0A22FA295AF70B0E090968C9137
:1055500090E02F7002C0959587952A95E2F780FD1F
:105560005EC0DB01CA01482A592A6A2A7B2A440FF5
:10557000551F661F771F8E169F0601F7F70131979B
:1055800080818F3F11F00E94001650EA5A95F1F782
:10559000F6014082518262827382F4E0CF0ED11C08
:1055A0002E143F0409F0A4CF48E150E0B80180EE8A
:1055B00093E00E948234FF24F394009709F4F12CC5
:1055C000892B89F188E1F801A0EEB3E001900D92FA
:1055D0008A95E1F781E08093A2030E948121909354
:1055E000A1038093A0038091A0039091A1030E9446
:1055F00072210597E0F0E0EEF3E0ADE4B4E088EF6F
:1056000093E041915191619171914D935D936D93AF
:105610007D938E179F07A9F71092A20308C080E020
:1056200090E0DC01A0CF8091A2038111DCCF8090BB
:10563000AE03082C000C9908AA08BB0810910001C1
:10564000212F30E081E090E0281739070CF0B2C03C
:105650006091AA037091AB038091AC039091AD036C
:105660000E94E9102B013C0145E6441651046104F7
:105670007104FCF08091A90390E0019662E370E070
:105680000E94F5338093A90382559C4FFC01108240
:10569000812F113308F080E38F5F809300010E9417
:1056A00005116093AA037093AB038093AC039093AE
:1056B000AD03F2E08F169104A104B1040CF489C08B
:1056C000A0E6BAEEA50194010E9457344B015C019B
:1056D00044E6149F90011124032E000C440B550B3B
:1056E000240D351D461D571DA5E0B0E00E9457341E
:1056F0009B01AC01C501B4010E94093449015A0162
:1057000051EF85169104A104B10428F080EF882E92
:10571000912CA12CB12C6091A5037091A6038091CE
:10572000A7039091A8030E94E9102B013C0185E694
:10573000481651046104710484F00E9405116093BD
:10574000A5037093A6038093A7039093A803809169
:1057500008048093A4038092A3031091A403A09152
:10576000A303A11BBB0BA30192010E94623424E698
:1057700030E040E050E00E942B34120F10930804F8
:105780008F2D68960FB6F894DEBF0FBECDBFDF91A8
:10579000CF911F910F91FF90EF90DF90CF90BF902E
:1057A000AF909F908F907F906F905F904F903F90C1
:1057B0002F900895FC01E255FC4F4081042E000C0F
:1057C000550B660B770B840E951EA61EB71E019611
:1057D0003BCF812C912C54019ECF1F921FB61F925C
:1057E00011248F939F93AF93BF9380919D059091C8
:1057F0009E05A0919F05B091A0054196A11DB11DE8
:1058000080939D0590939E05A0939F05B093A0055E
:10581000BF91AF919F918F911F901FBE1F901895C0
:10582000CDB7DEB7E0970FB6F894DEBF0FBECDBFA1
:1058300084B7877F84BF0FB6F894A89580916000E5
:10584000886180936000109260000FBE80E890E055
:105850000FB6F89480936100909361000FBE85B7F6
:10586000806885BF85B7806885BF8EEF95E190938E
:105870001903809318030E945A0F0E9425108091EB
:10588000E20084608093E20078948091CB058823C5
:10589000A1F01091E9001F709091EC00892F8170A8
:1058A00090FD80E8182B1092E9008091E80083FDBC
:1058B0000E94F5191F701093E90082E084BD93E007
:1058C00095BD9AEF97BD80936E000E94761F81115F
:1058D00002C00E94D21E00E511E046E5E42E41E040
:1058E000F42ED8018D918D018F3F11F00E9400168A
:1058F000E016F106B1F706E511E037E6E32E31E0F8
:10590000F32EF80181918F018F3F11F00E94001654
:10591000E016F106B1F788E1EDE4F4E0DF01282FAD
:105920001D922A95E9F7E0EEF3E0DF011D928A95DA
:10593000E9F70E94B81F811102C00E94C31F82E0D4
:1059400090E00E949F34809334040E948F1F9093B4
:10595000A2058093A1050E94462AEFE3FCE9319756
:10596000F1F700C000000E94462A80914D0480FF9C
:1059700008C06FEF7FEF90E080E00E94DB340E9470
:10598000EC1D83E090E00E949F340E9478180E94F2
:10599000B81F811104C00E94C31F0E949D1F46E0D2
:1059A00050E06CE170E08DED95E00E948F34109234
:1059B000DC058091DD058C7F11F40E949D1F0E9403
:1059C00081219093100480930F041092310480E899
:1059D0008093E4050E94CE326DE070E086EA92E1A9
:1059E0000E946D19892BE9F58091310463E070E024
:1059F00081FD78C183EA92E10E946D19892B89F5B6
:105A00006DE070E083E992E10E946D19892B49F500
:105A10000E940511605A75418F4F9F4F6093910509
:105A2000709392058093930590939405EDEEF5E0C5
:105A300080E092E0DF019C011D9221503040E1F7AF
:105A4000F093EE07E093ED078FEF9FEF9093EC0557
:105A50008093EB0581E080939605809395051092E5
:105A600032046091A10560686093A1051091A205C0
:105A700084E090E00E94BD34612F82E290E00E94B9
:105A8000BD3481E091E090939A05809399050E943E
:105A9000462A882E81110E9405112DE4222E24E031
:105AA000322E05E314E03CA62BA6B12CA12CABA50D
:105AB000BCA54D905D906D907D90BCA7ABA7F80103
:105AC00080819181A281B38184159505A605B705D2
:105AD00009F44FC09C01AD012425352546255725E5
:105AE0002DA73EA74FA758AB912CC12CD12C7601E6
:105AF000C3948DA59EA5AFA5B8A98C219D21AE21EB
:105B0000BF21892B8A2B8B2B61F199A2AAA221E0BC
:105B1000D301C2018C219D21AE21BF21892B8A2B6B
:105B20008B2B09F420E02BA30E9481218160782F28
:105B30009DA38CA349A15AA16BA18DA10E94B62956
:105B4000F80180819181A281B3818C259D25AE25AC
:105B5000BF2580839183A283B383B394FBE0FB15BD
:105B600000F19394CC0CDD1CEE1CFF1C21E1921281
:105B7000C0CFA3940C5F1F4F36E0A31298CFB11093
:105B800010C08FEF8EA38FA318A60E948121816081
:105B9000782F9AA789A74EA15FA168A58AA50E9420
:105BA000B6290E9405116093F8037093F90380935E
:105BB000FA039093FB033091DD05432F4370F42EDD
:105BC00019F0F32EF694F69420911B01213009F47C
:105BD0009AC0222309F489C0223009F481C12330FC
:105BE00009F487C180919605882309F4A6C260E074
:105BF00080E00E94A81180910F04909110040E94EF
:105C000072218838934108F095C180910E0481116A
:105C100091C183EB92E10E94EB0E2091EB05309154
:105C2000EC052115310509F46FC280913204811110
:105C30006BC2082F10E0AA24A394B12C082E02C036
:105C4000AA0CBB1C0A94E2F7A9014A215B21452B4F
:105C500009F4E3C29091310490FDE1C28295880F6E
:105C60008076809312019801369527953695279571
:105C700020931501815E809313011092160124E692
:105C800030E047E050E060E171E088E70E947D335A
:105C9000892B09F039C2A80165E0440F551F6A95A8
:105CA000E1F78091310480FDC8C243515A4F04E6A8
:105CB00010E020E230E060E488E70E94A433892B02
:105CC00009F022C20E94B819C50180959095A09054
:105CD000EB05B090EC05A822B922B092EC05A09299
:105CE000EB0512C280EA92E187CE10921801609310
:105CF000D5057093D6058093D7059093D80551E0CC
:105D000050931B016FCF90910E0181E0F9120BC0EF
:105D1000832F837020910D0130E091E082171306EC
:105D200009F490E0892F817080931A018091E20537
:105D300090911901981739F08093190140E060E0C3
:105D400080E00E9475128CE08F1578F0EF2DF0E066
:105D5000E953F94C0C944A3480911A01882341F19B
:105D600040E060E080E00E94751280E021C0009178
:105D7000180184E1089F002D112414E1E12EE00EAA
:105D8000DE2C94E69E1510F4B4E6DB2E6091DE0561
:105D90007091DF058091E0050E94E113C62EB72EB9
:105DA000A82E10E00D15C0F081E0A3E6AE15E8F2D4
:105DB000909118019F5F90931801811113CF82E099
:105DC00080931B0180911A0181110CCFF1100ACF31
:105DD00083E080931B0106CFF801EC54FD4F8081D6
:105DE00090911901892331F02A2D4C2D6B2DC8017A
:105DF0000E9477120F5F1F4FD5CF8EE593E10E946F
:105E0000B015D6CF85E593E1FACF8CE493E1F7CFD7
:105E10008EE393E10E94D714CBCF8FEA93E10E94E7
:105E20005415C6CF86E293E1FACF8BE093E1F2CF2F
:105E30008EED92E10E947514BBCF80EB92E1FACF18
:105E400089E792E1F7CF0091180184E1089F002DC6
:105E50001124A4E1EA2EE00EDE2CB4E6BE1510F407
:105E6000F4E6DF2EB090DF05C090E0051091DE056E
:105E70006091E1056695669566958091D50590914E
:105E8000D6050E94D7130E946013805887FD819524
:105E9000880F682F2CE0629F612D1124610F7B2DEC
:105EA0008C2D0E94E113C62EB72EA82E10E00D15E2
:105EB00030F081E0E3E6EE1508F07ACF56CFF80136
:105EC000EC54FD4F808190911901892331F02A2DE6
:105ED0004C2D6B2DC8010E9477120F5F1F4FE7CF2B
:105EE000F0920E01832F837080930D010E94101E8B
:105EF0006FCF8091DC05882351F046E050E06CE1E3
:105F000070E08DED95E00E94AD341092DC0560915B
:105F1000D5057091D6058091D7059091D8050E943E
:105F2000E910603171058105910508F45BCE10928E
:105F30001B0158CE21E020930E040E949C11D82E04
:105F400010910804612F70E090E080E00E94843599
:105F500020E030E040E250E40E9434369B01AC0186
:105F600060E070E081EE93E40E94E1342B013C019B
:105F700020E030E048EC52E40E944E3587FD13C12A
:105F8000C301B2010E945335609304047093050469
:105F90008093060490930704153108F409C10E9408
:105FA000B8196091000470910104809102049091ED
:105FB00003040E94E910009104041091050420914B
:105FC000060430910704061717072807390760F4FD
:105FD0000E940511609300047093010480930204F1
:105FE000909303040E9431190E9405116093FC03F1
:105FF0007093FD038093FE039093FF0360E08EE0B7
:106000000E94A81184ED94E10E946C1D4090080448
:1060100080910F01841105C080910D04803309F433
:1060200049C040920F0180E380930D04512C712CE4
:10603000612C10920C04C301B2012AE030E040E070
:1060400050E00E940934605D603331F04114510426
:106050006104710409F460E360930B0460E35AE0A7
:10606000451651046104710488F0C301B2012AE0AD
:1060700030E040E050E00E940934CA01B9012AE052
:1060800030E040E050E00E940934605D60930A0413
:1060900020E384E6481651046104710448F0C3010A
:1060A000B20124E630E040E050E00E940934205D77
:1060B00020930904E9E0F4E001900020E9F7DF0112
:1060C00011977D0109E014E00E151F0508F49FC02B
:1060D00062E081E10E94A8118AEC94E1D1FE02C045
:1060E0008FEC94E10E946C1D63E081E10E94A81195
:1060F00080EC94E1D2FE02C085EC94E10E946C1D1C
:1061000080919605811189CD809195058823A9F00C
:106110000E9405110091910510919205209193051F
:1061200030919405601B710B820B930B6F3F7F4F77
:106130008F4F9F4710F40E949D1981100E94B8193B
:106140000E949C1190913304891721F00E949C11A8
:10615000809333048091CB05843009F098CC83E0A0
:106160008093E9008091E80082FF91CC8091E80063
:1061700090E085FF06C00E94790F882309F4C0C013
:1061800091E08091E8008B778093E800992309F4EF
:106190007ECCE981E150E33108F02BC1F0E0EC5214
:1061A000F94C0C944A3464E670E080E090E0ECCE68
:1061B0006091FC037091FD038091FE039091FF03B9
:1061C0000E94E91061367A4E8105910518F00E940F
:1061D0009D1914CF60910004709101048091020414
:1061E000909103040E94E9106D3271408105910580
:1061F00008F404CF0E940511609300047093010419
:1062000080930204909303040E943119F7CEF801A1
:1062100081918F010E94BE1C57CF8F5F0ACD880FDE
:10622000880F880F8093120110921501895F809367
:10623000130183E08093160122CD80E2A1E1B4E056
:106240001D928A95E9F7EBE6F1E0FCA7EBA767E67C
:1062500071E037E0E32EABA5BCA52D91BCA7ABA7A1
:10626000FB014190BF01440E552E511CC2018351C8
:106270009A4F2C01E22FF0E0EF5EFB4F90E080E0C0
:10628000CE2CC81AFF24F394082E01C0FF0C0A94E8
:10629000EAF7320100E0D3011D913D011F212C2DB1
:1062A000201B2770D22E022E000C330BB12F01C001
:1062B000BB0FDA94EAF7DB2E31952195310927706F
:1062C000332701C016952A95EAF7D12A1081D12AE1
:1062D000D0820F5F0830F9F601963196883091052B
:1062E00079F6EFE6F1E02BA53CA5E217F30709F0FC
:1062F000B2CF04E610E020E230E041E154E0DBCC34
:1063000000E210E0AE014F5F5F4F7A018091E8003C
:1063100085FD0AC08091E8008B778093E8000E9499
:10632000790F882399F32CCF8091F100D7018D93B9
:106330007D010150110951F723CF1A8289E08B8327
:1063400011C08A81823009F420C1833091F18130FB
:1063500009F04FC00E9405110E9450346B837C836A
:106360008D839E838091CB05843009F090CB109172
:10637000E9001F709091EC00892F817090FD80E8FA
:10638000182B82E08093E9008091E80080FF0DC027
:1063900050E040E060E270E0CE0101960E94AA0F5A
:1063A0008091E8008E778093E8001F701093E900D9
:1063B0006ECBFE013196D1014D915D916D917D9134
:1063C0001D016283538344833396B5E62B16B4E0F4
:1063D0003B0689F7C7CF8A81823059F46B817C8173
:1063E0008D819E810E94503486E290E00E94BD34EF
:1063F000B9CF8FEF8983B6CF4C816B818A810E94A0
:10640000E11E9827892798279E838D83ABCFED8047
:10641000FE80FE24EF24FE248A810B81E2E20E9F9F
:1064200080011124FCEC8F9F000D111D11248C8123
:1064300090E0880F991F080F191F6F2DC8018796CC
:106440000E94BD346E2DC8018896D0CF0E94641E74
:1064500089CF80E18A8386CF82E08A8381E46FCF0F
:10646000CA80DB80DC24CD24DC248E010F5F1F4F2B
:10647000EC80E00EF12EF11CC60181549E4FE01617
:10648000F10609F46FCF21E4C21622E0D20658F4D7
:106490000E949F34D80114968C93FFEFCF1ADF0A25
:1064A0000F5F1F4FE9CFF8011482F7CF0A811B81DC
:1064B0001027012710279E012F5F3F4F6901EC80B5
:1064C000E00EF12EF11CC80181549E4FE016F1063A
:1064D00009F448CF013432E0130728F4D6011496AA
:1064E0006C910E94BD34BFEFCB1ADB0A0F5F1F4FC8
:1064F000EACF0E94541E36CF82E0ACCFCA80DB8048
:10650000DC24CD24DC248E010F5F1F4FEC80E00ED5
:10651000F12EF11CC60187960E151F0509F422CF36
:10652000E8E9CE16E1E0DE0658F40E949F34D80177
:1065300014968C93FFEFCF1ADF0A0F5F1F4FEACF3D
:10654000F8011482F7CF0A811B8110270127102739
:106550009E012F5F3F4F6901EC80E00EF12EF11C90
:10656000C80187960E151F0509F4FCCE083931E0E5
:10657000130728F4D60114966C910E94BD34BFEF26
:10658000CB1ADB0A0F5F1F4FEBCF86E290E00E9431
:106590009F341B821C821D828E83E4CE1092B90030
:1065A0008CE08093B80008959F92AF92BF92CF92F3
:1065B000DF92EF92FF920F931F93CF93DF93B82E4A
:1065C000EB010E9481216C01EE24E394F12CC43193
:1065D000D10560F025E0E22EF12CCF3FDC0731F051
:1065E000CE0164E170E00E94D5337B0184EAA82EDD
:1065F00094E8992E1092BC00A092BC000E948121C8
:106600008C018091BC0087FF0DC08091B900887F0C
:10661000883039F18091B900887F803111F10FEF16
:106620001FEF09C00E948121801B910B8E159F05D1
:1066300040F30EEF1FEFCF3FDC07E1F2C6010E94EF
:1066400072218C179D07B0F2C801DF91CF911F9185
:106650000F91FF90EF90DF90CF90BF90AF909F9001
:106660000895B092BB009092BC000E9481218C01E1
:106670008091BC0087FF0AC08091B900887F883173
:1066800011F0803461F610E000E0DECF0E9481213D
:10669000801B910B8E159F0558F3CBCF0F931F9343
:1066A000CF93DF93EB018093BB0084E88093BC0021
:1066B0000E9481218C018091BC0087FF11C0209134
:1066C000B900287F81E090E0283211F490E080E06A
:1066D000919581959109DF91CF911F910F91089527
:1066E000CF3FDC0741F30E948121801B910B8C1767
:1066F0009D0708F38EEF9FEFEECFCF92DF92EF92E0
:10670000FF920F931F93CF93DF936B018A0179015F
:10671000B9010E94D432E6010C0D1D1DC017D1072E
:1067200061F424E92093BC00DF91CF911F910F9178
:10673000FF90EF90DF90CF90089597FDF2CFB701D3
:1067400089910E944E33EACFCF92DF92EF92FF926F
:106750000F931F93CF93DF93C62F6A017901B8017E
:106760000E94D43297FD0CC0B8018C2F0E944E338A
:10677000E601EC0CFD1CCE15DF0511F097FF0CC0F7
:1067800024E92093BC00DF91CF911F910F91FF90DE
:10679000EF90DF90CF900895B80189910E944E3319
:1067A000EACF84E98093BC000895AA1BBB1B51E18A
:1067B00007C0AA1FBB1FA617B70710F0A61BB70B71
:1067C000881F991F5A95A9F780959095BC01CD0116
:1067D0000895991B79E004C0991F961708F0961B3D
:1067E000881F7A95C9F78095089597FB072E16F4B0
:1067F000009407D077FD09D00E94D53307FC05D05F
:106800003EF4909581959F4F0895709561957F4FC7
:106810000895A1E21A2EAA1BBB1BFD010DC0AA1FE1
:10682000BB1FEE1FFF1FA217B307E407F50720F0F9
:10683000A21BB30BE40BF50B661F771F881F991F74
:106840001A9469F760957095809590959B01AC01BD
:10685000BD01CF010895052E97FB1EF400940E9400
:10686000423457FD07D00E94093407FC03D04EF490
:106870000C94423450954095309521953F4F4F4FA1
:106880005F4F089590958095709561957F4F8F4FDC
:106890009F4F0895EE0FFF1F0590F491E02D09948E
:1068A00069279627692778278727782708950E94E0
:1068B0006A34A59F900DB49F900DA49F800D911DEB
:1068C00011240895B7FF0C9457340E945734821B4B
:1068D000930B0895A29FB001B39FC001A39F700DB9
:1068E000811D1124911DB29F700D811D1124911DD8
:1068F0000895FB01DC0102C005900D92415050400B
:10690000D8F70895FB01DC0104C08D910190801936
:1069100021F441505040C8F7881B990B0895DC01C1
:10692000CB01FC01F999FECF06C0F2BDE1BDF89A9A
:10693000319600B40D9241505040B8F70895F9993E
:10694000FECF92BD81BDF89A992780B50895A8E140
:10695000B0E042E050E00C949134DC01A40FB51F8C
:106960004150504048F0CB01840F951F2E910E945A
:10697000BE3441505040D0F70895262FF999FECFEC
:1069800092BD81BDF89A019700B4021639F01FBA82
:1069900020BD0FB6F894FA9AF99A0FBE089503969F
:1069A000272F0E94BE340E94BD34252F0E94BE3482
:1069B000242F0C94BE340196272F0E94BE340C94D1
:1069C000BD345058BB27AA270E94F9340C94FA35DD
:1069D0000E94EC3538F00E94F33520F039F49F3FE7
:1069E00019F426F40C94E9350EF4E095E7FB0C94C9
:1069F000E335E92F0E940B3658F3BA176207730785
:106A00008407950720F079F4A6F50C942D360EF442
:106A1000E0950B2EBA2FA02D0B01B90190010C01AE
:106A2000CA01A0011124FF27591B99F0593F50F4C6
:106A3000503E68F11A16F040A22F232F342F44271E
:106A4000585FF3CF469537952795A795F040539516
:106A5000C9F77EF41F16BA0B620B730B840BBAF0E6
:106A60009150A1F0FF0FBB1F661F771F881FC2F751
:106A70000EC0BA0F621F731F841F48F48795779565
:106A80006795B795F7959E3F08F0B0CF9395880F1F
:106A900008F09927EE0F9795879508950E94BF35C6
:106AA00008F481E008950E94133688F09F5798F00B
:106AB000B92F9927B751B0F0E1F0660F771F881F03
:106AC000991F1AF0BA95C9F714C0B13091F00E941D
:106AD0002D36B1E008950C942D36672F782F882736
:106AE000B85F39F0B93FCCF3869577956795B39544
:106AF000D9F73EF490958095709561957F4F8F4FB3
:106B00009F4F0895E89409C097FB3EF490958095B7
:106B1000709561957F4F8F4F9F4F9923A9F0F92F63
:106B200096E9BB279395F695879577956795B795E1
:106B3000F111F8CFFAF4BB0F11F460FF1BC06F5FC7
:106B40007F4F8F4F9F4F16C0882311F096E911C0D9
:106B5000772321F09EE8872F762F05C0662371F0FA
:106B600096E8862F70E060E02AF09A95660F771F0E
:106B7000881FDAF7880F9695879597F90895990FEA
:106B80000008550FAA0BE0E8FEEF16161706E807F7
:106B9000F907C0F012161306E407F50798F0621B18
:106BA000730B840B950B39F40A2661F0232B242BED
:106BB000252B21F408950A2609F4A140A6958FEF0C
:106BC000811D811D089597F99F6780E870E060E05E
:106BD00008959FEF80EC089500240A941616170676
:106BE00018060906089500240A94121613061406BE
:106BF00005060895092E0394000C11F4882352F021
:106C0000BB0F40F4BF2B11F460FF04C06F5F7F4FD8
:106C10008F4F9F4F089557FD9058440F551F59F0BF
:106C20005F3F71F04795880F97FB991F61F09F3F79
:106C300079F087950895121613061406551FF2CFA2
:106C40004695F1DF08C0161617061806991FF1CFF2
:106C500086957105610508940895E894BB27662719
:106C60007727CB0197F908950E9447360C94FA359F
:106C70000E94EC3538F00E94F33520F0952311F096
:106C80000C94E3350C94E93511240C942E360E94B3
:106C90000B3670F3959FC1F3950F50E0551F629F1F
:106CA000F001729FBB27F00DB11D639FAA27F00D65
:106CB000B11DAA1F649F6627B00DA11D661F829F8C
:106CC0002227B00DA11D621F739FB00DA11D621F71
:106CD000839FA00D611D221F749F3327A00D611D8E
:106CE000231F849F600D211D822F762F6A2F112470
:106CF0009F5750409AF0F1F088234AF0EE0FFF1FA3
:106D0000BB1F661F771F881F91505040A9F79E3FF9
:106D1000510580F00C94E3350C942E365F3FE4F37C
:106D2000983ED4F3869577956795B795F795E7954F
:106D30009F5FC1F7FE2B880F911D9695879597F958
:106D40000895F894FFCFDB1A031BA61C031BA61C97
:106D5000361B571BA61C551C621C611F611F6A1F36
:106D60006A1F6C1F6A1F6A1F6A1F611F611F711FE4
:106D70006A1F6A1F711F88258825DF25DF251026D9
:106D8000BB25BB25BB252A269B26AB26AB26AC2ED6
:106D9000B72EFD2E022F052F082F0D2F122F152F86
:106DA000182F1D2F202F232F9D31A131EB31FC31C6
:106DB00007322632F931F931F931F931F931293215
:0E6DC0002C323032563279327C327E32A3329F
:106DCE0001E610AC1DE510A81DA41DE410FFFFFF89
:106DDE000021007F2200030100FF000300FFC88195
:106DEE008283E200E900EA00B500B600B700CD00EC
:106DFE008301CC008A019201940121022302240214
:106E0E002502260227022A02B300B4006F0070008A
:106E1E00303132333795F0F1F4F5F6F76636353416
:106E2E0097969467C69293000810181810080000E1
:106E3E003131295A1B750A40226D3B011901AC00F4
:106E4E008717A017C01757565554535251504F4ECF
:106E5E004D4C4BFF4A49483738393A3B3C3D3E3F53
:106E6E004041424344454647363534333231302F64
:106E7E002E2D2C2B2A29282726191A1B1C1D1E1FC6
:106E8E002021222324FF25FFFFFF181716151413A8
:106E9E001211100F0E0D0C0BFF0AFF000102FFFF67
:106EAE0003FFFFFFFF040506FF070809014013401B
:106EBE00254058409140A340B540C640D340E040E5
:106ECE00D334B932AB2D9134843477346A345D3493
:106EDE0050344334363429341C34123200320028F4
:106EEE00152922292F293C29492956296329702938
:106EFE007D298A299729B02AE01DD31DC61DAD1BF9
:106F0E00A21D951D881D7B1D6E1D611D541D471DE7
:106F1E003A1D2D1D201D131D031D00110D111A11DB
:106F2E002711341141114E115B1168117511821127
:106F3E008F119C11AF11C611D311E011E000D300D7
:106F4E00C600B600A9009C008F007B006E00610099
:106F5E0054004100340027001A00000001063206DA
:106F6E0059068706B006C606DD37C03A8A3B603D35
:106F7E002A3B073C01010104010101040404040140
:106F8E0001040404040404040404040401080404B5
:106F9E0004040404040404040401040404040404A6
:106FAE000404040404040404040401040404040496
:106FBE000404040404040404010404040408040482
:106FCE00040404040404040404040401020202027E
:086FDE0002020202020202029B
:00000001FF
